:020000040800F2
:1000000068060020D5010008DD010008DF010008B6
:10001000E1010008E3010008E5010008000000001C
:10002000000000000000000000000000E7010008E0
:10003000E901000800000000EB010008ED010008E4
:10004000EF010008EF010008EF010008EF010008D0
:10005000EF010008EF010008EF010008EF010008C0
:10006000EF010008EF010008EF010008EF010008B0
:10007000EF010008EF010008EF010008EF010008A0
:10008000EF010008EF010008EF010008EF01000890
:10009000EF010008EF010008EF010008EF01000880
:1000A000EF010008EF010008EF010008EF01000870
:1000B000EF010008EF010008EF010008EF01000860
:1000C000EF010008EF010008EF010008EF01000850
:1000D000EF010008EF010008EF010008EF01000840
:1000E000EF010008EF010008EF010008EF01000830
:1000F000EF010008EF010008EF010008EF01000820
:10010000EF010008EF010008EF010008EF0100080F
:10011000EF010008EF010008EF010008EF010008FF
:10012000EF010008EF010008EF010008EF010008EF
:1001300000F002F800F03AF80AA090E8000C8244BF
:100140008344AAF10107DA4501D100F02FF8AFF29C
:10015000090EBAE80F0013F0010F18BFFB1A43F0A5
:1001600001031847D0040000F0040000103A24BF37
:1001700078C878C1FAD8520724BF30C830C144BF0C
:1001800004680C607047000000230024002500264E
:10019000103A28BF78C1FBD8520728BF30C148BFEA
:1001A0000B6070471FB51FBD10B510BD00F035F8CE
:1001B0001146FFF7F7FF00F021FA00F053F803B4FF
:1001C000FFF7F2FF03BC00F05BF8000080F3088843
:1001D000704700000948804709480047FEE7FEE7EE
:1001E000FEE7FEE7FEE7FEE7FEE7FEE7FEE7FEE7E7
:1001F00004480549054A064B70470000E904000819
:100200003101000868000020680600206802002014
:1002100068020020704770477047754600F02CF860
:10022000AE4605006946534620F00700854618B0E3
:1002300020B5FFF7DDFFBDE820404FF000064FF08E
:1002400000074FF000084FF0000B21F00701AC460B
:10025000ACE8C009ACE8C009ACE8C009ACE8C0092A
:100260008D46704710B50446AFF300802046BDE8C8
:100270001040FFF7A4BF00000048704704000020B2
:1002800001491820ABBEFEE72600020070470000BF
:100290000149C860704700000020024030B50446A4
:1002A00004254FF4302000F089F80546042D17D1BD
:1002B0000C48006940F002000A49086108464461A0
:1002C000006940F0400008614FF4302000F076F8FB
:1002D00005460448006941F6FD710840014908617E
:1002E000284630BD0020024004200B49C96801F0B7
:1002F000010109B101200EE00749C96801F00401BC
:1003000009B1022007E00449C96801F0100109B1F0
:10031000032000E0042070470020024004200B4925
:10032000C96801F0010109B101200EE00749C9685F
:1003300001F0040109B1022007E00449C96801F095
:10034000100109B1032000E00420704700200240A2
:100350000348006940F080000149086170470000CF
:100360000020024070B504460D460426F00200F05D
:1003700025F80646042E11D10948006940F0010015
:10038000074908612580F00200F018F80646044885
:10039000006941F6FE71084001490861304670BDB0
:1003A0000020024002480349486003484860704703
:1003B0002301674500200240AB89EFCD00B502461E
:1003C0000423FFF791FF034603E0FFF78DFF034689
:1003D000521E012B01D1002AF7D102B9052318467C
:1003E00000BD10B502460B460020002100BF04E00E
:1003F00032F811400444A0B2491C9942F8D310BD10
:1004000010B500F001F810BD0CB50020019000906F
:100410003348006840F480303149086000BF3048FC
:10042000006800F4003000900198401C0190009892
:1004300018B90198B0F5A06FF1D12948006800F40F
:10044000003010B10120009001E0002000900098E1
:10045000012843D12348006840F01000214908607A
:100460000846006820F0030008600846006840F075
:10047000020008601A484068194948600846406808
:1004800048600846406840F480604860084640681C
:1004900020F47C1048600846406840F4E81048604A
:1004A0000846006840F08070086000BF0C48006893
:1004B00000F000700028F9D00948406820F00300DF
:1004C000074948600846406840F00200486000BFA5
:1004D0000348406800F00C000828F9D10CBD00006A
:1004E000001002400020024010B51348006840F0A0
:1004F00001001149086008464068104908400E494B
:100500004860084600680E4908400B4908600846E4
:10051000006820F4802008600846406820F4FE004F
:1005200048604FF41F008860FFF76AFF4FF00060DB
:100530000449086010BD0000001002400000FFF8F0
:10054000FFFFF6FE08ED00E070B548E04FF4A03183
:100550002748FFF746FF4FF6FF7188422FD1FFF77C
:1005600021FF3520FFF794FE00240AE0214901EB2A
:10057000C420FFF793FE00BFFFF7D0FE0128FBD099
:10058000641C502CF2D31C480668002413E0184960
:1005900031F8145000BFFFF7C1FE0128FBD0154908
:1005A00001EB44002946FFF7DDFE00BFFFF7B6FE72
:1005B0000128FBD0641CB442E9D3FFF7C9FEFFF762
:1005C000F1FE3520FFF764FE0B48801EFFF766FE44
:1005D00000BFFFF7A3FE0128FBD0FFF7B9FE0648D6
:1005E000801E00884AF6AA218842AFD070BD000064
:1005F00000A002080020000802F00708FFF7A4FF8F
:1006000011E00948006809490840B0F1005F0AD1CB
:10061000054840680649086003490868FFF7D6FDA9
:10062000034800688047ECE7002000080000FE2F28
:100630000000002054060008000000200400000014
:100640006C01000858060008040000206406000041
:08065000880100080000000011
:0400000508000131BD
:10200000603500204521000845430008353E0008A2
:10201000D94100084D350008257200080000000075
:10202000000000000000000000000000256E000815
:102030009138000800000000472A00087955000880
:102040005F2100085F2100085F2100085F21000870
:102050005F2100085F2100085F2100085F21000860
:102060005F2100085F2100085F2100085F21000850
:102070005F2100085F2100085F2100085F21000840
:102080005F2100085F2100085F2100085F21000830
:102090005F2100085F2100085F2100085F21000820
:1020A0005F2100085F2100085F2100085F21000810
:1020B0005F2100085F2100085F2100085F21000800
:1020C0005F2100085F2100085F2100085F210008F0
:1020D0005F210008A97100085F2100085F21000846
:1020E0005F2100085F2100085F2100085F210008D0
:1020F000BD6F00085F2100085F2100085F21000814
:102100005F2100085F2100085F2100085F210008AF
:102110005F2100085F2100085F2100085F2100089F
:102120005F2100085F2100085F2100085F2100088F
:10213000DFF80CD000F02CFC00480047F5900008B8
:10214000603500200648804706480047FEE7FEE766
:10215000FEE7FEE7FEE7FEE7FEE7FEE7FEE7FEE757
:10216000616E00083121000872B6704762B6704790
:10217000EFF3108072B6704780F31088704730BF5D
:10218000704720BF7047B0FA80F0704790FAA0F017
:10219000B0FA80F0704790FAA0F07047F0B480EA8F
:1021A0000102D40F4200B2EB410F02D202460846B0
:1021B00011464A0042D0C30DDDB2C1F3C752AD1A79
:1021C000202D35DAC1F3160141F4000204B1524268
:1021D000C5F1200602FA06F12A411044B3EBD05FA4
:1021E00023D0C4B1012DA0EBC35009DCF0BC4FF0EB
:1021F000004202EAC352DBB200F5000000F00DBB62
:10220000400000F1807000EBC350A0F1807040EA04
:10221000D170490009E0490841EAC071A0EBC35000
:1022200000F50000400800EBC350F0BC00F0ECBA31
:102230006142012202EB4101001BF6E7F0BC70474E
:1022400081F00041AAE780F00040A7E780EA0102A0
:1022500010B502F00043400022D04A001FD0010E0A
:1022600001EB1261C0F35600C2F3560240F40000C5
:1022700042F40002A0FB022000047F39140400D0C5
:10228000401C50EA124001D44000491EC2B20C0664
:1022900004EBD010401C4008802A02D003E000204C
:1022A00010BD20F00100002900DA0020184310BD05
:1022B00030B480EA010202F0004530F0004221F023
:1022C000004013D090B1C30DD40DC2F31601C0F37A
:1022D0001600E41A41F4000140F400027D349142FA
:1022E00001D3641C00E04900002C02DA30BC00205D
:1022F00070474FF400000023914201D3891A034331
:1023000040084FEA4101F7D151B1914202D14FF05B
:10231000004105E002D24FF0010101E06FF0010140
:1023200003EBC450284430BC00F06EBA2DE9FE4FD8
:10233000804681EA0300C00F0C46009021F0004166
:1023400023F00045B8EB0200A94105D240462146E2
:1023500090461C460B46024623F00040104347D0EF
:10236000270DC7F30A00C3F30A510290401A0190E7
:1023700040286BDAC3F3130040F4801B00989246A8
:1023800020B10023D2EB030A63EB0B0B01985946F3
:10239000C0F14002504600F016FA06460D4650467F
:1023A0005946019A00F01EFA10EB08006141002422
:1023B00087EA115284EAE7731A4340D0009A62B365
:1023C000019A012A4FEA075215DC001B61EB02015A
:1023D0004FF0004202EA0752CDE90042001C41F5ED
:1023E000801132462B4600F055FA03B0BDE8F08F5D
:1023F00040462146F9E7001B61EB0201001C41F554
:10240000801300185B412018A2F5001747EB030169
:1024100040EAD570B6196D4111E06D084FEA3606F5
:1024200045EAC0754FEA0752001B61EB0201001C30
:1024300041F5801149084FEA3000001951413246F8
:102440002B4603B0BDE8F04F00F015BA009801220A
:1024500040000023D0EB020263EBE07300982146BA
:102460004FEAE074B8EB000061EB0401E9E783F0A8
:1024700000435BE781F0004158E72DE9FE4F81EA18
:10248000030404F0004421F0004100944FF0000BDD
:1024900023F0004350EA01045ED052EA03045BD00B
:1024A000C3F30A54C1F30A552C44A4F2F334019443
:1024B000A0FB0254C1F3130141F48011C3F31303D1
:1024C00043F4801301FB024400FB034E840A970A85
:1024D00044EA815447EA8357A4FB076802958D0AB2
:1024E00005FB07854FEA932C04FB0C542705029D3E
:1024F0004FEA065847EA1637B5EB08056EEB070CAE
:10250000870E920E47EA811742EA8312A7FB020167
:10251000B6EB0B0164EB00042B0D43EA0C335E18A1
:1025200044EB1C50DA465146E7FB0201C5F31304A5
:102530004FEA0B3343EA14534FEA0432019C43EA57
:102540000603A4F10C040294009CCDE900B400F051
:10255000A1F903B0BDE8F08F00200146F9E72DE9AD
:10256000F04D81EA030404F0004B21F000451446CD
:102570004FF0000A23F0004150EA050220D054EA4F
:1025800001021DD0C5F30A570246C5F31303C1F378
:102590001300C1F30A5640F4801543F48013A7EBEF
:1025A0000608101BD64608F2FD3873EB050002D36F
:1025B00008F1010801E092185B41B8F1000F03DA5D
:1025C00000200146BDE8F08D00204FF48011064642
:1025D00084460EE0171B73EB050705D3121B63EB54
:1025E000050306434CEA010C49084FEA30009218F3
:1025F0005B4150EA0107EDD152EA030012D082EAB2
:10260000040083EA0501084305D0101BAB4106D244
:102610000122002306E000224FF0004302E06FF0A9
:10262000010253101AEB06004CEB085110EB0A00A4
:1026300041EB0B01BDE8F04D00F01DB9C10F80EA80
:10264000E0700844CA079623002100F0E6B89623FC
:102650000022114600F0E1B800F0004220F00040F6
:10266000C10DC0F3160040F400007F2901DA0020FC
:102670007047962903DCC1F19601C84001E0963904
:102680008840002AF4D04042704720F00040C10D3D
:10269000C0F3160040F400007F2901DA00207047E3
:1026A000962903DCC1F19601C840704796398840ED
:1026B000704700F0004230F000400AD0C10D01F533
:1026C0006071C0F3160042EA0151C208400711438D
:1026D000704700200146704701F0004330B421F0FC
:1026E000004150EA010206D00A0DA2F56072C1F362
:1026F0001301002A02DC30BC00207047440F44EA7A
:10270000C104C100E01830BC00EBC25000F07CB83E
:10271000002801DBC0F10040002901DBC1F10041CC
:1027200081427047002801DBC0F10040002901DB35
:10273000C1F100418842704730B50B460146002088
:102740002022012409E021FA02F59D4205D303FA73
:1027500002F5491B04FA02F52844151EA2F10102F4
:10276000F1DC30BD2DE9F05F0546002092469B4626
:1027700088460646814640241BE028464146474697
:10278000224600F017F953465A46C01A914110D319
:1027900011461846224600F016F82D1A67EB01087C
:1027A0004F4622460120002100F00DF817EB0009EA
:1027B0004E41201EA4F10104DFDC484631462A4682
:1027C0004346BDE8F09F202A04DB203A00FA02F1DC
:1027D000002070479140C2F1200320FA03F319430F
:1027E00090407047202A06DBCB17203A41FA02F0CE
:1027F00043EAE07306E041FA02F3D040C2F120025E
:1028000091400843194670470029A8BF7047401CF3
:10281000490008BF20F00100704710B4B0FA80FCF6
:1028200000FA0CF050EA010404BF10BC704749B133
:10283000CCF1200421FA04F411FA0CF118BF0121A3
:1028400021430843A3EB0C01CB1D4FEA00614FEA83
:10285000102042BF002010BC704700EBC350104452
:102860000029A4BF10BC7047401C490008BF20F0DD
:10287000010010BC704710B5141E73F1000408DA93
:10288000401C41F1000192185B411A4301D120F034
:10289000010010BD2DE9F04D92469B4611B1B1FAF1
:1028A00081F202E0B0FA80F220329046FFF78BFF0F
:1028B00004460F4640EA0A0041EA0B0153465A46D5
:1028C000084313D0114653EA010019D0C8F1400261
:1028D000504600F06FF805460E46504659464246AF
:1028E000FFF771FF084305D0012004E02046394678
:1028F000BDE8F08D0020054346EAE0762C433743DF
:102900000A986305E40AA0EB08000022FD0A44EAE5
:1029100047540A3002D500200146E9E701051019A5
:102920006941DDE9084500196941BDE8F04DA2E7BC
:10293000C1F30A52C1F3130140F2FF3341F4801195
:102940009A4202DA00200146704740F233439A422D
:10295000A2F2334202DC524200F02CB8FFF733BF40
:1029600030B5041E71F1000404DB4FF00044404216
:1029700064EB0101141E73F1000405DB1C464FF0EB
:102980000043524263EB0403994208BF904230BDBA
:10299000064C074D06E0E06840F0010394E80700AC
:1029A00098471034AC42F6D3FFF7C6FB94A4000856
:1029B000B4A40008202A04DB203A21FA02F0002106
:1029C000704721FA02F3D040C2F12002914008433F
:1029D0001946704730B58C1810F8012B12F00F0310
:1029E00001D110F8013B120906D110F8012B03E0C8
:1029F00010F8015B01F8015B5B1EF9D101E001F801
:102A0000013B521EFBD1A142E6D3002030BD0000A5
:102A10001D484FF0FF010170002080F309881B481A
:102A2000016881F308881A484FF08051016062B64E
:102A3000FEE717484FF080510160704714484FF08F
:102A400080510160704772B6EFF3098028B12038D9
:102A500080E8F00F0F490968086000B50E4880470C
:102A60005DF804EB0D480E490A78027009480D49DB
:102A70000A680260106890E8F00F203080F309883F
:102A80004EF0F40E62B6704722ED00E00400002024
:102A900004ED00E0BC000020095400084A000020BA
:102AA0004B000020C000002070B500F071FD04460E
:102AB000032C03D0042C01D0022C0ED1052005F0EC
:102AC00005FF06464449FFF7F3FB0546FFF7DDFD2A
:102AD00081B24248A0F85A1303E000213F48A0F811
:102AE0005A13002005F0F2FE06463B49FFF7E0FBD3
:102AF0000546FFF7CAFD3949A1F85003012005F04A
:102B0000E5FE06463449FFF7D3FB0546FFF7BDFD5A
:102B100081B23248A0F85213022005F0D7FE0646D3
:102B20002D49FFF7C5FB0546FFF7AFFD81B22B48E6
:102B3000A0F85413032005F0C9FE054601F092F8F1
:102B40002649A1F85603042005F0C0FE054601F011
:102B500089F82249A1F85803062005F0B7FE064679
:102B60001F49FFF773FB0546FFF78FFD81B21B4836
:102B7000A0F85C1300201B49088048808880C8802A
:102B8000088148811548B0F8440388811348B0F89B
:102B90004603C8811148B0F8500308820F48B0F8C6
:102BA000520348820D48B0F8540388820B48B0F8AD
:102BB0005603C8820948B0F8580308830748B0F89C
:102BC0005A0348830548B0F85C0388830348B0F88B
:102BD0005E03C88370BD000000002041641900201E
:102BE0000000C8425C2600201CB501F01FF8104808
:102BF000104908601AE0104A6946002001F0EEFA18
:102C000070B9BDF800200D490B4803F0D9FF044608
:102C10000A4A2146002001F039FB094804F072F904
:102C200001AA00214FF4FA7002F01EFCE3E7000055
:102C30008C260020D4000020EA280020162A00203C
:102C40007019002008B5002405F016FA15E0601C84
:102C500084B20A480078012805D00A2C06DB00243B
:102C600006F078FA02E0002406F074FA05F000FAA3
:102C70006A460021642002F0F7FBE8E7C400002068
:102C800010B5012005F0E8F9012004490870002082
:102C90000349088001200349087010BD6E0100201F
:102CA000700100207201002010B52749C86827492B
:102CB000FFF738FD01D8012000E0002004461CB9D0
:102CC00000202349087002E00120214908702148B2
:102CD0004078022807D01F484078032803D01D48B9
:102CE0004078042802D10220194908701848007859
:102CF00020B1012809D0022824D10DE0002005F0E0
:102D0000ABF90020144908801CE0012005F0A4F96B
:102D100000201149088015E00F480088401C0E492A
:102D20000880084600881E280BDB002008800B481E
:102D3000007880F00100094908700846007805F025
:102D40008BF900BF00BF10BD7821002000409C45DA
:102D50006E010020EC0000207001002072010020B4
:102D600010B50D49486A0D49FFF7D2FC05D2012282
:102D700011020B4806F0AAF80CE00749486A4FF028
:102D80008241FFF7CFFC05D200224FF48071044846
:102D900006F09CF810BD0000782100200000A04043
:102DA0000010014010B540F20A6006F049FC022014
:102DB00006F064FB002005F025F800210C4804F023
:102DC000C6FF012211460A4804F09EFF4FF460221C
:102DD0000121074804F0F3FF01221146044804F0E2
:102DE000CFFF034804F0C3FF014804F078FF10BD93
:102DF0000028014010B502230E2200210C4805F0E6
:102E00000FF801210A4805F065F800BF02210848C3
:102E100004F0F0FF0028F9D00221054804F0E7FF94
:102E2000034805F053F80446FFF711FC10BD0000FD
:102E30000028014010B5AB22134B1B681A71062203
:102E4000114B1B685A71B1F5967F1BD800220E4BAF
:102E50001B681A8011E00C4A12681288835C0A4AC7
:102E60001268921D084C246824881355064A12687B
:102E70001288521C044B1B681A80034A126812887D
:102E80008A42E8D310BD0000D4000020F8B5044603
:102E90000026164801780078401C144A1070012959
:102EA00022DB0020114608706B460022902110485A
:102EB00001F038F80646BEB99DF80150BDF8000093
:102EC000000200B20090BDF8000000F47F4000B2A4
:102ED0000090BDF9000028430090BDF90000C11723
:102EE00000EB116109122180F8BD0000D80000201C
:102EF000F82F002010B50021014807F07EF810BD22
:102F00000034014010B50548807800B110BD0121A2
:102F1000034807F072F800BFF8E70000EC0000205B
:102F2000003401402DE9F041184908681849FFF7BD
:102F3000EFFB02D80020BDE8F0811648808940F6FA
:102F400048514843050B2846FFF778FB8046124955
:102F5000FFF77CF90646114801681148FFF776F93A
:102F600007463146FFF71AF90C4908604FF07C51CB
:102F70000A480068FFF712F90646FFF76DFB0446A2
:102F8000002C00DA00242046D5E70000782100203C
:102F900000803B46103000200AD7A33C900100205F
:102FA00048E17A3F2DE9F05F404908684049FFF762
:102FB000AFFB02D80020BDE8F09F3E4800883D49A5
:102FC0004988884201DA002505E03A4800883949F5
:102FD0004988401A05B240F648506843800A04B256
:102FE000322C00DA00243448007878B9002004E05C
:102FF000324921F81040411CC8B20828F8DBE00033
:103000002F49086001202C49087017E02B482D49F2
:10301000097830F911002A490968081A2849086016
:1030200026482849097820F811402649097830F9BE
:1030300011002349096808442149086021480078A3
:10304000401C2049087008460078082801DB002051
:1030500008701B490868C11700EB5171C9100FFABD
:1030600081F84046FFF7EAFA834617480168584658
:10307000FFF7E6F882461549FFF7E8F8814612485F
:1030800001684846FFF78AF806460F4806604FF089
:103090007C513046FFF782F88146FFF7DDFA07469C
:1030A000002F00DA0027384685E70000782100204D
:1030B00000803B4610300020880100201E30002098
:1030C00084010020800100208C0100200AD7A33C4D
:1030D0000448C08840F648514843000B00EB4000CC
:1030E00080007047103000200448408940F6485165
:1030F0004843000B00EB4000800070471030002078
:103100000448808840F648514843000B00EB4000DB
:1031100080007047103000200448008940F6485174
:103120004843000B00EB4000800070471030002047
:1031300010B500F0BBF800F01BF800F081F8FFF7C5
:1031400031FE00F02DF910BD10B54FF400410248DA
:1031500005F0B8FE10BD00000008014010B54FF4A6
:103160000041024805F0B0FE10BD0000000801401B
:1031700010B540F2096006F063FA022006F07EF90D
:10318000002004F03FFE002202212C4804F0B1FE92
:1031900001221102294804F0ACFE0021274804F066
:1031A000D6FD07220121254804F0AEFD03230022AD
:1031B0001146224804F034FE0323012211461F4821
:1031C00004F02EFE0323022211461C4804F028FEC0
:1031D00003231A461946194804F022FE0323042249
:1031E0001146164804F01CFE03230522114613481D
:1031F00004F016FE032306221146104804F010FEC8
:103200004FF4602201210D4804F0D9FD012211463E
:103210000A4804F0B5FD094804F0A4FD074804F08D
:10322000A6FD4FF47A7005F039F9044804F057FD13
:103230000121024804F04EFE10BD000000240140B0
:1032400000B587B04FF4A06006F0FAF900211448E9
:1032500005F03CFA1348009000208DF81800124841
:10326000029001208DF81900000201908000039067
:1032700000208DF81A00072004904FF400500590AC
:103280006A460021064805F059FA0021044805F075
:10329000CEF90021024805F098F907B000BD000002
:1032A000000002404C2401401030002010B540F2D4
:1032B000026006F0C5F940F2036006F0C1F940F281
:1032C000046006F0BDF940F2056006F0B9F94FF46C
:1032D000C06006F0B5F94023012218212C4805F002
:1032E00053FE802301221821294805F04DFE80233A
:1032F00001221821274805F047FE01231A4618210C
:10330000254805F041FE0121244805F0A3FE4FF4B5
:103310000043012210211F4805F036FEFFF714FF7D
:103320000223012210211A4805F02EFE0123042257
:103330000021184805F028FE022304220021154828
:1033400005F022FE04231A460021124805F01CFE57
:103350000823042200210F4805F016FE1023042242
:1033600000210C4805F010FE20230422002109480A
:1033700005F00AFE102304220021054805F004FE92
:10338000402304220021034805F0FEFD10BD00008B
:103390000010014000080140000C01400002300014
:1033A00000B58BB040F20D6006F04AF9464806F0D1
:1033B00049FD0020ADF810004020ADF812000020BB
:1033C000ADF8140040F22B1006900020ADF8160066
:1033D0008DF81C0004A93C4806F0A8FD0120ADF8BA
:1033E00020000420ADF822000020ADF82400ADF844
:1033F0002600ADF82800ADF82A0008AA00213248BE
:1034000006F08EFB08AA01212F4806F089FB08AAC6
:1034100003212D4806F084FB1D2200212A4806F0D6
:10342000A2FC60220021284806F070FC082200213E
:10343000254806F0ABFC1D220121234806F093FC31
:1034400070220121204806F061FC082201211E485B
:1034500006F09CFC642203211B4806F084FC7022C9
:103460000321194806F052FC0020ADF80000ADF829
:1034700002000C20ADF804000020ADF80600ADF805
:103480000800ADF80A00ADF80C0069460E4806F0D9
:1034900038FB01210C4806F0B0FD20210A4806F057
:1034A000A4FD0121084806F08DFD012200212C20F9
:1034B00005F062FE044806F01FFB05F039FC0248E7
:1034C00006F02EFD0BB000BD0034014010B5022304
:1034D0000A2200210C4804F0A3FC01210A4804F050
:1034E000F9FC00BF0221084804F084FC0028F9D050
:1034F0000221054804F07BFC034804F0E7FC044685
:10350000FFF7A5F810BD00000028014010B5022308
:103510000D2200210C4804F083FC01210A4804F02C
:10352000D9FC00BF0221084804F064FC0028F9D04F
:103530000221054804F05BFC034804F0C7FC044684
:10354000FFF785F810BD00000028014000BFFEE72E
:1035500030B502460B46002100244FF6FF7000BF35
:1035600012E0555C684000240AE000F0010525B136
:1035700040104AF20105684000E04010651CACB202
:10358000082CF2DB4D1CA9B29942EADB30BD0000E9
:103590000148407870470000EC00002010B5FFF7AC
:1035A000C7FD00200149487010BD0000EC0000205C
:1035B0000149487070470000EC00002010B5FFF78B
:1035C000A1FCFFF7CBFD10BD10B5FFF793FCFFF793
:1035D000BBFD10BD70B56248407806287ED2DFE89A
:1035E00000F0B403071625AA00205E49C862B0E0C7
:1035F0005D480078022805D001205C490870002051
:103600005B4908604FF4C8705649C862A1E056484B
:103610000078032805D0012054490870002054493F
:1036200008604FF47A704F49C86292E04E480078C3
:10363000042826D04B498868FFF70EF80446FEF7A9
:10364000FDFF4C49486147498868FFF705F8044683
:10365000FEF7F4FF4749C86148690021FFF758F8B1
:1036600002D2002043494861424948694249FFF774
:1036700059F802D240483F49486100203F4948611B
:10368000C8613849C868FEF7E7FF0446224647F29A
:103690004811384803F0D8FD3249C8623749C86933
:1036A0003749FFF73FF834D82E49C86AFEF7C6FFFE
:1036B00005463449FEF7CAFD04462A48816820467B
:1036C000FFF730F825D2274988682F49FEF7BEFD5D
:1036D0000546FEF7C1FF0446224800E035E0C06A17
:1036E000A04201DA1F48C46A322C00DA32241D4895
:1036F000C4622046FEF7A2FF05461E4841692846DF
:10370000FFF706F804D22046FEF798FF19494861F2
:1037100000BF1448C06AB0F57A7F04DD4FF47A70B8
:103720001049C86206E00F48C06A002802DA00208B
:103730000C49C8620DE000200E494861C8610F497C
:103740004861C8610749C86203E000200549C862B2
:1037500000BF00BF024840780349087070BD0000F8
:10376000EC00002078210020A5010020E0000020CE
:10377000E40000203001002000007A44F400002022
:103780003333733FCDCC4C3FCDCC8C3F2DE9F0474C
:1037900004460E46174639463046FEF751FD81462F
:1037A0003A494846FEF784FD804641462068FEF7C8
:1037B0004DFD0546206AFEF741FF8246E169FEF7AE
:1037C000A7FF07D2606AFEF739FF8246E169FEF77C
:1037D000A9FF19D3206AFEF731FF8246E169FEF79F
:1037E000A1FF04D800214046FEF79CFF0CD3606A7D
:1037F000FEF724FF8246E169FEF78AFF0DD800211B
:103800004046FEF785FF08D241466068FEF71EFD80
:1038100082466169FEF7C2FC6061E06AFEF70EFF56
:1038200082466169FEF774FF03D2E06AFEF706FF85
:103830006061A06AFEF702FF82466169FEF772FFCF
:1038400003D2A06AFEF7FAFE606128466169FEF7BE
:10385000A5FC0546606AFEF7F1FE82462946FEF7A2
:1038600057FF03D2606AFEF7E9FE0546206AFEF7BD
:10387000E5FE82462946FEF755FF03D2206AFEF791
:10388000DDFE0546E5612846BDE8F0870000FA4404
:103890007047000010B505F085F940F2053005F0DD
:1038A0008DF84FF4417005F089F840F2023005F0D0
:1038B00085F8002411E00D4901EBC42005F000F962
:1038C00040F2053005F07AF84FF4417005F076F8D3
:1038D00040F2023005F072F8641C502CEBD304481F
:1038E00005F0EEF805F0D6F810BD000000A00208C3
:1038F00000F007082DE9F04106466948807850B984
:103900006748407838B166484078012803D0644859
:103910004078052803D105F07FFFBDE8F0816149BB
:10392000486AFEF78BFE07463146FEF7F1FE04D2E9
:103930005C49486AFEF782FE064600213046FEF7E3
:10394000E7FE00D200265848007840B100205649D2
:1039500008704FF07E56534948613046C861504860
:10396000007830B1012813D0022825D003287DD15A
:1039700090E04E4A1168D068FEF79AFC0446214652
:103980003046FEF763FC0446204605F0C7FE84E09F
:10399000464AD1681068FEF78BFC07464FF07E510F
:1039A000FEF751FC054629463046FEF74FFC05461A
:1039B000284605F075FE70E03C4A1168D068FEF7B5
:1039C00077FC044600253A492046FEF7ABFE11D2AB
:1039D000374C364908682146FEF738FC80463348A4
:1039E000C1684046FEF764FC07464FF07E51FEF783
:1039F0002AFC05464FF07E513046FEF789FE01D283
:103A0000304601E04FF07E5007462146FEF71EFC8F
:103A100004464FF07E513046FEF784FE0FD24FF041
:103A20007E513046FEF70CFC80462249FEF70EFC24
:103A3000074639462846FEF7B1FB054604E029460D
:103A40003046FEF703FC05461A492846FEF76AFE93
:103A500000D2184D16492046FEF764FE00D2144CE1
:103A600015492046FEF754FE02D200E011E0124C48
:103A700010492846FEF756FE00D20E4D002128467A
:103A8000FEF746FE00D200252946204605F076FEC8
:103A900003E000BF05F0C0FE00BF00BF00BF3CE771
:103AA000EC000020F40000206D01002078210020AF
:103AB0003333733FAE47613E6666263F10B55948C3
:103AC00000780A2802DB002056490870FFF70CFB3B
:103AD0000446FEF7B3FD53490A78091D41F8220058
:103AE000081F0078401C091F0870084690F82C0039
:103AF0000A2802DB002081F82C00FFF70DFB0446AA
:103B0000FEF79CFD0146474890F82C20303040F8E5
:103B10002210303890F82C00401C424981F82C00CB
:103B2000084690F858000A2802DB002081F8580067
:103B3000FFF7CEFA0446FEF781FD0146394890F8BA
:103B400058205C3040F822105C3890F85800401C37
:103B5000344981F85800084690F884000A2802DBAE
:103B6000002081F884003048416A2E4890F8842073
:103B7000883040F82210883890F88400401C294989
:103B800081F88400084690F8B0000A2802DB002083
:103B900081F8B0002449B1F92800FEF74FFD014635
:103BA000204890F8B020B43040F82210B43890F893
:103BB000B000401C1B4981F8B000084690F8DC00BA
:103BC0000A2802DB002081F8DC00FFF7EBF904464D
:103BD000FEF734FD0146134890F8DC20E03040F851
:103BE0002210E03890F8DC00401C0E4981F8DC001F
:103BF000084690F808010A2802DB002081F8080135
:103C000000F0B0FA0146074890F8082100F58670E8
:103C100040F82210034890F80801401C014981F83F
:103C2000080110BD041800207821002073210C48E1
:103C3000A0F84213B0F842034FF6FF7101EA0021E9
:103C40000748A0F8441347F21E41A0F84613B0F805
:103C5000460300F47F400249A1F84003704700008A
:103C60006419002070B505460D492846FEF7EEFAA6
:103C7000064600212846FEF755FD04D83046FEF7DB
:103C800004FD84B20AE031460020FEF7D9FA064668
:103C90003046FEF7FAFC84B244F40044204670BD7E
:103CA0000000C8422DE9F04704460025FFF7A2F8BE
:103CB000804641464FF08B40FEF7C2FA81460A49E2
:103CC0004046FEF7C3FA82464946FEF7F1FA074638
:103CD0000649FEF7EDFA06462146304600F008F8A0
:103CE0002846BDE8F087000000401C4600007A44EA
:103CF0002DE9F05F83468A463C495846FEF708FDA9
:103D00000AD83B495846FEF7A1FA04463949FEF75E
:103D100045FACAF8000066E034495846FEF702FD4D
:103D20000FD235495846FEF7F3FC0AD833495846B6
:103D3000FEF78CFA04463249FEF730FACAF8000062
:103D400051E02D495846FEF7EDFC18D22D49584652
:103D5000FEF7DEFC13D85846FEF7ABFC80462A4A35
:103D60002A4BFEF78AFB06464FF00042284BFEF72F
:103D7000DDFA0446FEF7B0FCCAF8000033E0214942
:103D80005846FEF7CFFC0FD222495846FEF7C0FC3A
:103D90000AD821495846FEF759FA04461F49FEF74A
:103DA000FDF9CAF800001EE01A495846FEF7BAFCB1
:103DB0000FD21B495846FEF7ABFC0AD819495846A2
:103DC000FEF744FA04461849FEF7E8F9CAF800007D
:103DD00009E016495846FEF739FA04461449FEF739
:103DE000DDF9CAF80000BDE8F09F00009A999940FB
:103DF000B0031CC19358B4420000204113F271C0BB
:103E0000E9A67642CDCC644164CC5D4BC88700C046
:103E1000E9A646403333B3418885A2BFDB79064229
:103E20000000E441D34D62BF1D5AC9414F1EB6BECA
:103E3000DD24EC4000BFFEE770B504460025A18AF2
:103E4000206905F03FF82189606805F03DF8012000
:103E500004F024FBA18A206905F036F8032004F061
:103E60001DFB2189606805F0EDF8012800D10125CE
:103E7000A18A206905F026F8012004F00FFB2846EE
:103E800070BD70B504460D46A18A206905F01AF888
:103E9000012004F003FB2189606805F015F800207B
:103EA0002870072620E0A18A206905F00BF8012080
:103EB00004F0F4FAA18A206905F006F8032004F062
:103EC000EDFA2189606805F0BDF8012803D1297851
:103ED000B04001432970A18A206904F0F3FF022059
:103EE00004F0DCFA701E46B2002EDCDA70BD10B5AC
:103EF0000446A18988B205F0A3FBA38A01221421FC
:103F0000206905F041F8238901221421606805F039
:103F10003BF82189606804F0D7FFA18A206904F08A
:103F2000D3FF10BD2DE9F84380460E4617461C46C8
:103F300000250020208006F0FE06404600F0ADF887
:103F40003146404600F03EF84046FFF775FF00B1AD
:103F50006D1E3946404600F035F84046FFF76CFFCD
:103F600000B16D1E46F00106404600F096F831465D
:103F7000404600F027F84046FFF75EFF00B16D1E97
:103F800069464046FFF77DFF20889DF800100843F2
:103F90002080404600F049F869464046FFF771FF2F
:103FA00020889DF800104FF47F4202EA0121084367
:103FB0002080404600F055F8404600F086F828463C
:103FC000BDE8F8832DE9F04104460E460127072598
:103FD00027E0A18A206904F075FF012004F05EFA51
:103FE00046FA05F000F0010020B12189606804F074
:103FF0006BFF03E02189606804F064FF012004F096
:104000004DFAA18A206904F05FFF052004F046FA0A
:10401000A18A206904F056FF012004F03FFA681ECF
:1040200045B2002DD5DABDE8F08110B50446A18A6D
:10403000206904F047FF2189606804F043FF0120F4
:1040400004F02CFAA18A206904F03EFF052004F058
:1040500025FAA18A206904F035FF012004F01EFA38
:1040600010BD10B50446A18A206904F02BFF2189F8
:10407000606804F029FF012004F010FAA18A206989
:1040800004F022FF052004F009FAA18A206904F057
:1040900019FF012004F002FA10BD10B50446218971
:1040A000606804F011FF022004F0F8F9A18A206989
:1040B00004F00AFF022004F0F1F92189606804F09D
:1040C00001FF022004F0EAF910BD10B50446A18AF0
:1040D000206904F0F7FE012004F0E0F9218960680E
:1040E00004F0F0FE012004F0D9F9A18A206904F05F
:1040F000EBFE022004F0D2F92189606804F0E4FEAE
:10410000012004F0CBF910BD2DE9F04180460D46A9
:1041100016461F46002405F0FE054046FFF7BDFF8A
:1041200029464046FFF74EFF4046FFF785FE00B1A7
:10413000641E31464046FFF745FF4046FFF77CFED0
:1041400000B1641E39464046FFF73CFF4046FFF78A
:1041500073FE00B1641E4046FFF7B7FF2046BDE87E
:10416000F08100002DE9FE4F4FF0000AD3460020F9
:104170000290FFF7CBF98246FFF7A8F98346514634
:104180005846FEF7CFFA1BD251465846FEF758F86C
:104190004FF08B410090FEF78BF80190FEF789FA03
:1041A00080464FF06632094BFEF767F90646084A2B
:1041B000084BFEF7D4F90446FEF78EFA029001E0B0
:1041C000002002900298BDE8FE8F000066660A405B
:1041D0004C37894160E5C03F00BFFEE72DE9F04163
:1041E00004460E4690460025274850F824000079E2
:1041F000AB2842D1244850F824004179224850F895
:1042000024004079401C204A52F82420507106298D
:1042100038DB56201C4951F82410087100201A4937
:1042200051F824104871184850F824000088308054
:104230000020154951F8241008803188124A52F89C
:104240002420901DFFF784F90746DFB900BF0EE078
:104250000D4850F82400801D405D08F80500FF213E
:10426000094850F82400801D4155681C85B23088EB
:10427000A842EDDC0020BDE8F0810020024951F8A1
:10428000241048710120F6E7D40000202DE9F04702
:1042900004460E4690464FF00009002E4BDDB6F561
:1042A000957F48DC002509E018F80510234850F8F0
:1042B000240000F599704155681C85B2B542F3DBC6
:1042C0001E4951F8241001F599703146FFF740F965
:1042D00007461A4850F8240000F5997087553A0AA5
:1042E000164850F8240000F59970711C425404BB24
:1042F000B01C1FFA80F9002518E0104850F824007F
:1043000090F83201012806D100BF07210C4805F0C2
:104310006EFF0028F9D0094850F8240000F5997084
:10432000415D074805F007FF681C85B24D45E4DB99
:1043300000E000BF00BF4846BDE8F087D400002081
:10434000003801407047000010B5002807DA0A075E
:10435000140E054A00F00F031B1FD45403E00A0794
:10436000130E024A135410BD18ED00E000E400E003
:104370007047000010B50348006810B1014800689C
:10438000804710BD1C00002070B5044600F0A2F864
:1043900000203E4908703E4908703E4908703E4979
:1043A00008603E4908603E4908703E4908703E4931
:1043B00008703E48006858B13D48056845B13B4823
:1043C000066803E0761E002028602D1D002EF9D11E
:1043D0000020384908603849086038490860384981
:1043E0000860384908603849086038490860384929
:1043F000087001F05FFC01F099FC204601F0ACF977
:10440000208800B170BD204601F00CFA208800B170
:10441000F8E7204601F012FA208800B1F2E72046C2
:1044200001F08CFA208800B1ECE7204601F072FC24
:10443000208800B1E6E7204601F00CFD208800B19D
:10444000E0E7204601F03AFF208800B1DAE7204695
:1044500001F0B0F9208800B1D4E7204602F032FA2A
:10446000208800B1CEE7204601F072FE208800B11E
:10447000C8E7204602F08AFA208800B1C2E701F0BE
:1044800097F8FFF775FF00BFBCE700003000002081
:104490003100002056000020BC000020C000002099
:1044A0004A0000204B0000204C000020C8A2000859
:1044B000C4A20008100000201400002018000020F2
:1044C0001C000020200000202400002028000020E4
:1044D00082000020064800680649096800EB810058
:1044E000054908600846006820F00700086070472A
:1044F000C4A20008C8A200080400002010B50024CF
:104500002D480078012800D010BD00BFFDF730FE17
:10451000044600BF2948007828B900BF2046FDF7AF
:104520002BFE00BFF0E725480078401E23490870A5
:1045300008460078002805DD00BF2046FDF71CFE78
:1045400000BFE1E71E480078002805DD00BF2046D7
:10455000FDF712FE00BFD7E701F098FB194908707C
:104560000846007800EB4000174951F82000174931
:1045700008600846006816490968884205D100BFEE
:104580002046FDF7F9FD00BFBEE710480068D0F8EF
:104590008400401C0D490968C1F884000D4800687A
:1045A000401C0C490860FEF749FA00BF2046FDF7A1
:1045B000E3FD00BF00BFA7E731000020300000206E
:1045C000560000204B000020BC120020C00000203C
:1045D000BC000020780000202DE9F04104460E4682
:1045E000154600271B480078002804DD42F6E160EC
:1045F0002880BDE8F0811CB945F6C3502880F8E753
:1046000000BF00BFFDF7B4FD074600BF00BF124862
:10461000206066600020206284F82500A0624020AF
:1046200084F8240004F1080001F03FFA204601F06C
:104630006DF90A480088401C0849088000BF00BF87
:104640003846FDF799FD00BF00BF0020288000BF5D
:10465000CFE70000300000204D555458480000209E
:104660002DE9F04788B00546894690461C46109EC5
:104670004FF0000A8A480078002805DD46F2AE10A7
:10468000308008B0BDE8F0871DB945F6C3503080D2
:10469000F7E7B8F1000F03D0B8F5004F02D100E002
:1046A00000BF03E045F625603080EAE700BF7D49A2
:1046B0002868884203D045F6C4503080E1E70CB149
:1046C0000020206000BF00BFFDF752FD824600BF02
:1046D00000BF95F82500C0B9734800682862724889
:1046E000006890F8370085F82400012085F825003F
:1046F0000CB1A86A206000BF00BF5046FDF73CFD2A
:1047000000BF00BF00203080BBE76749286A096806
:10471000884212D195F82500401C85F825000CB17F
:10472000A86A206000BF00BF5046FDF725FD00BF0E
:1047300000BF45F282703080A3E708F4004050B11A
:1047400000BF00BF5046FDF717FD00BF00BF46F297
:10475000B010308095E75548007800280ADD00BF8A
:1047600000BF5046FDF708FD00BF00BF46F663508E
:10477000308086E72F6A97F837004B49096891F82F
:10478000371088423ADD97F8360008282AD2DFE849
:1047900000F004151E1F17162021384601F02CFBCF
:1047A0004148006890F8370087F8370097F83700DD
:1047B00001F08CFA384601F0E1FA1EE000BF00BFBC
:1047C0003948006890F8370087F8370015E000BFD7
:1047D00000BF00BF3448006890F83710384601F039
:1047E00041F90AE000BF00BF5046FDF7C5FC00BF1D
:1047F00000BF46F62D60308043E700BF4B460422E1
:104800002946684601F0A6F800BF00BF5046FDF7F4
:10481000B3FC00BF00BF00F003F900BF00BFFDF70D
:10482000A7FC824600BF00BF1F48006890F8350013
:1048300030B101280CD002281AD0032821D110E071
:104840001CB119480068006C2060002030801CE01A
:104850001CB115480068006C206046F2A910308039
:1048600013E00CB10020206047F2D92030800CE02A
:104870001CB10D480068006C206045F6C2503080C5
:1048800003E046F62E60308000BF00BF00BF00BFCF
:104890005046FDF771FC00BF00BF00BFF1E600000D
:1048A000300000204D555458BC0000205600002018
:1048B0002DE9F84F04460F4615464FF0000A5448BC
:1048C0000078002804DD46F20E202880BDE8F88F2D
:1048D0001CB945F6C3502880F8E71FB1B7F5004F63
:1048E00002D100E000BF03E045F625602880EDE737
:1048F00000BF48492068884203D045F6C45028804C
:10490000E4E700BF00BFFDF733FC824600BF00BFF5
:104910004149206A096888420AD000BF00BF50465A
:10492000FDF72AFC00BF00BF45F281702880CDE76B
:104930004FF000092534C4F803902078401E207001
:1049400014F8250900280ADD00BF00BF5046FDF716
:1049500013FC00BF00BF45F283702880B6E704F166
:104960000808B8F8080068B90020206284F825001B
:1049700000BF00BF5046FDF7FFFB00BF00BF002097
:104980002880A3E72448006890F8370094F82410A2
:10499000884219D02048006801F02EFA94F82400CB
:1049A0001D49096881F837001B49096891F83700EB
:1049B00001F08CF91848006801F000FA1648006808
:1049C00090F8370015490870D8F80000866826620C
:1049D00096F8370084F82400012084F8250000238D
:1049E0001A4631462046CDF8009001F0CFF800BFBE
:1049F00000BF5046FDF7C0FB00BF00BF07F40040FA
:104A000008B900F00DF80020288000BF5EE7000024
:104A1000300000204D555458BC0000204A000020B2
:104A200010B500241F480078002800DD10BD1E4886
:104A30000078002800DDF9E700BFFDF799FB044688
:104A400000BF01F023F9194908700846007800EB0F
:104A50004000174951F820001649086008460068D0
:104A600015490968884205D100BF2046FDF784FB3F
:104A700000BFDBE70F480068D0F88400401C0D49F8
:104A80000968C1F884000D480068401C0B490860A3
:104A9000FDF7CFFF00BF2046FDF76EFB00BF00BF54
:104AA000C4E7000030000020560000204B0000202A
:104AB000BC120020C0000020BC00002078000020B4
:104AC00070B50446002517480078002803DD46F637
:104AD0006250208070BD14480078012803D045F64C
:104AE00089602080F6E711480078FA2803DB45F258
:104AF00009202080EEE700BF00BFFDF739FB054627
:104B000000BF00BF09480078401C0849087000BF7A
:104B100000BF2846FDF730FB00BF00BF002020800B
:104B200000BFD7E7300000203100002056000020F1
:104B300070B5044600251F480078002803DD46F6BE
:104B40006550208070BD1C480078012803D045F6D0
:104B500089602080F6E71948007818B946F6645055
:104B60002080EFE700BF00BFFDF702FB054600BF56
:104B700000BF12480078401E1049087008460078AF
:104B800000280ADD00BF00BF2846FDF7F5FA00BF88
:104B900000BF46F663502080D4E700BF00BF284620
:104BA000FDF7EAFA00BF00BFFFF73AFF00202080C0
:104BB00000BFC7E730000020310000205600002071
:104BC00010B5044612480078E8B901F05FF81149C1
:104BD000087008460078104908700E48007800EB0D
:104BE00040000E4951F820000D4908600846006851
:104BF0000C490860012006490870FDF709FF43F6DB
:104C00009920208002E045F68A60208010BD0000D7
:104C1000310000204B0000204A000020BC12002080
:104C2000C0000020BC0000202DE9F04107464FF0F5
:104C3000000800BF00BFFDF79BFA804600BF00BF21
:104C400000203849088038490860384908603849E8
:104C500008603849088100BF00BF4046FDF78CFA64
:104C600000BF00BF00BF00BFFDF782FA804600BF53
:104C700000BF3148046800BF00BF4046FDF77CFA22
:104C800000BF00BF1DE000BF00BFFDF771FA804606
:104C900000BF00BF002044F86C0F2063A061A08219
:104CA000E0826062A06220626C3C04F15806B08130
:104CB000D4F8AC4000BF00BF4046FDF75DFA00BF2E
:104CC00000BF002CDFD100BF00BFFDF751FA8046C6
:104CD00000BF00BF1948056800BF00BF4046FDF790
:104CE0004BFA00BF00BF12E000BF00BFFDF740FA63
:104CF000804600BF00BF05F120060020B081AD69ED
:104D000000BF00BF4046FDF737FA00BF00BF002DCF
:104D1000EAD101F0F3FC01F0DFFE00203880BDE8AD
:104D2000F081000062000020740000208800002054
:104D3000AC000020B01200207C00002050000020B9
:104D400010B50348006810B101480068804710BDE5
:104D5000200000202DE9FF4F85B004469046DDE994
:104D60001995159F139E002002905C48007800283A
:104D700005DD47F24A10288009B0BDE8F08F1CB964
:104D800047F2AD102880F7E7B8F1000F03D147F2E2
:104D90004F102880F0E71EB946F62F602880EBE719
:104DA0004F480068874203D246F630602880E3E728
:104DB0001498B84203D346F631602880DCE7129895
:104DC000402803D346F273202880D5E712983F2865
:104DD00006D14448844203D046F273202880CBE7B2
:104DE000204601F07BFA0020288009F0010088B1FC
:104DF00009F0020070B1B3460020049007E00020E3
:104E0000CBF800000BF1040B0498401C04900498AC
:104E1000B842F4D3149806EB80000390CDE90079F2
:104E200032464046039B089900F08CFA8346C4F84A
:104E300028800898E06206982062129884F837006B
:104E4000C4F800B00398A060189860606662A76319
:104E5000A4F83C904FF0000A08E0002104F1700033
:104E600040F82A100AF1010000F0FF0ABAF1000F21
:104E7000F3D004F15800169900F040FD204600F0F0
:104E800037F800BF00BFFDF773F9029000BF00BF05
:104E900094F8370000F01AFF204600F08FFF2046FC
:104EA00001F0D2F910480088401C0F4908800F48D3
:104EB0000078012807D000BF00BF0298FDF75CF919
:104EC00000BF00BF58E700BF00BF0298FDF754F9CC
:104ED00000BF00BFFFF7A4FD00BF4DE7300000207A
:104EE000F4A20008FC110020800000203100002006
:104EF00010B504460348006818B120460149096806
:104F0000884710BD1000002070B504460D460026ED
:104F100043480078002803DD47F24E10288070BD1A
:104F20004048844203D147F24C102880F7E77CB90F
:104F300000BF00BFFDF71CF9064600BF00BF3A489E
:104F4000046800BF00BF3046FDF716F900BF00BF80
:104F500000BF00BFFDF70CF9064600BF00BF94F884
:104F6000360008282DD2DFE800F004090E10080AE8
:104F70000F11204600F040FF2EE02DE000BF20463C
:104F800001F090FB28E000BF00BF00BF94F83400A0
:104F9000082810D2DFE800F004070508090A0B060C
:104FA00000BF00BF08E000BF00BF00BF00BF204639
:104FB00000F0B3FD00E000BF00BF204601F072FB2F
:104FC0000AE000BF00BF3046FDF7D6F800BF00BFC3
:104FD00046F62D602880A2E700BF04F1580000F0DB
:104FE0006BFC204600F024F8204601F045F90F48FC
:104FF0000088401E0D490880204601F06FF9FF200F
:1050000084F8360000BF00BF3046FDF7B5F800BF9A
:1050100000BF00202880FFF703FD00BF7FE70000EE
:1050200030000020FC110020BC0000208000002087
:1050300010B504460348006818B1204601490968C4
:10504000884710BD1400002010B5044603480068CE
:1050500018B1204601490968884710BD1800002092
:105060002DE9F04780460E4614461D464FF00009D4
:105070006D480078002805DD46F2AE10288000203B
:10508000BDE8F0871EB1B6F5004F02D100E000BFC9
:1050900004E045F6256028800020F1E700BF0CB150
:1050A0000020206000BF00BFFDF762F8814600BF0E
:1050B00000BF5E480068406C98B35C480068406C74
:1050C000401E5A490968486458480068476C1CB13A
:1050D00056480068006C206054480068006C4042EC
:1050E00052490968C1F8980050480068D0F89C00FF
:1050F0004E490968D1F89810884207D24B48006899
:10510000D0F8980049490968C1F89C0000BF00BF69
:105110004846FDF731F800BF00BF00202880384620
:10512000AEE7FFE706F4004058B100BF00BF4846B5
:10513000FDF722F800BF00BF46F2B0102880002023
:105140009EE73B48007800280BDD00BF00BF4846C3
:10515000FDF712F800BF00BF46F66350288000201C
:105160008EE7434607220021084600F0F3FB00BF0C
:1051700000BF4846FDF700F800BF00BFFFF750FC36
:1051800000BF00BFFCF7F4FF814600BF00BF274807
:10519000006890F8350020B1012824D0032832D1CE
:1051A0002AE0ECB121480068006C20601F480068CC
:1051B000006C40421D490968C1F898001B4800680E
:1051C000D0F89C0019490968D1F89810884207D294
:1051D00016480068D0F8980014490968C1F89C0086
:1051E0000020288013E01CB110480068006C20608B
:1051F00046F2A91028800AE00CB10020206047F296
:10520000D920288003E046F62E60288000BF00BF2A
:1052100006480068476C00BF00BF4846FCF7ACFF7B
:1052200000BF00BF38462BE730000020BC00002044
:10523000560000202DE9F04107460D4614461DB1E9
:10524000B5F5004F02D100E000BF05E045F625604E
:1052500020800020BDE8F08100BF002623463246B2
:105260002946384601F09AF880464046F2E70000A9
:105270002DE9F04705460E4617461C464FF0000A3A
:105280002E480078002804DD47F259102080BDE840
:10529000F0871EB946F2D5202080F8E71FB946F204
:1052A000D5202080F3E700BF00BFFCF761FF8246F6
:1052B00000BF00BF0DB922480568286868B900BF63
:1052C00000BF5046FCF758FF00BF00BF0020306011
:1052D000386047F252102080D9E795F83C0000F082
:1052E000010068B900BF00BF5046FCF745FF00BF92
:1052F00000BF00203060386047F254102080C6E7BD
:1053000000BF00BF5046FCF737FF00BF00BF4FF0A3
:105310000008D5F8249003E009F1040908F1010818
:10532000D9F800000028F7D0C6F80080A86BA0EBE1
:10533000080038600020208000BFA8E7300000206F
:10534000BC000020F0B50446DDE9055602EB8500FF
:1053500020F007004FF0807C071F3846C7F800C0D8
:10536000071F38463C60DFF89CC0071F3846C7F867
:1053700000C04FF0123C071F3846C7F800C04FF07E
:10538000033C071F3846C7F800C04FF0023C071F18
:105390003846C7F800C0071F38463B60071F38462D
:1053A00039604FF0113C071F3846C7F800C04FF076
:1053B000103C071F3846C7F800C04FF0093C071FD4
:1053C0003846C7F800C04FF0083C071F3846C7F8FA
:1053D00000C04FF0073C071F3846C7F800C04FF029
:1053E000063C071F3846C7F800C04FF0053C071FB2
:1053F0003846C7F800C04FF0043C071F3846C7F8CE
:1054000000C0F0BD8563000810B51448006810B1F5
:105410001248006880470024114800681149096853
:10542000884215D00E480068D0F88C00201A0C492C
:105430000968C1F888000A480068D0F89000084957
:105440000968D1F88810084405490968C1F8900036
:1054500004480068C0F88C4010BD00002400002003
:10546000BC000020C00000202DE9F04105460E469A
:105470001446002727480078002804DD47F27520ED
:105480002080BDE8F08124480078002803DD46F63E
:1054900063502080F5E736B1022E05D0042E0AD0E5
:1054A000082E09D101E000BF00BF1DB947F27E20E0
:1054B0002080E6E704E003E045F625602080E0E791
:1054C00000BF00BF00BFFCF753FE074600BF00BF90
:1054D0002346324629461148006801F085F82088A5
:1054E00038B100BF00BF3846FCF746FE00BF00BF22
:1054F000C7E70A48006800F07FFC00BF00BF3846DD
:10550000FCF73AFE00BF00BFFFF78AFA00202080B8
:1055100000BFB6E73000002056000020BC0000208D
:1055200008B500F01FF86A4600210A48FFF782FE1E
:1055300009480068401E084908600846006838B9F4
:105540000648006808606A4600210548FFF772FEB9
:1055500008BD000070160020B8000020B400002034
:105560005017002010B50348006810B101480068CA
:10557000804710BD2800002010B5002400BF00BFE8
:10558000FCF7F6FD044600BF00BF08480078401C49
:105590000649087000BF00BF2046FCF7EDFD00BFC4
:1055A00000BFFFF7BDFFFEF7A9FF10BD30000020D0
:1055B000244A2549254A264A2649274A2748284A6F
:1055C000284A294A294A2A482A482B4A2B482C4A41
:1055D0002C482D4A2D482E482E482F482F4A304A15
:1055E000304A3148314A324A3248334833483448E5
:1055F000344835483548364A364A374A374A3848B3
:1056000038483948394A3A4A3A4A3B483B483C4884
:105610003C493D483D4A3E4A3E4A3F4A3F4A404A4D
:10562000404A4148414A424A42484348434A444A20
:105630004448454A454A4648464800BF00BF00BF67
:10564000704700002CA3000890A400082DA30008B8
:105650002EA3000830A3000834A3000838A30008D4
:1056600035A3000860A3000861A3000862A3000836
:1056700064A3000866A300086AA300086CA30008DE
:105680008CA300088EA3000890A3000892A3000832
:1056900094A3000896A3000898A30008C4A30008D8
:1056A000C5A30008C6A30008C8A30008CAA3000831
:1056B000CBA30008CCA30008CEA30008D0A3000809
:1056C000D2A30008D4A30008D6A30008D8A30008DA
:1056D00008A4000809A400080AA400080BA40008F4
:1056E0000CA400080EA4000810A4000838A40008A8
:1056F00039A400083AA400083BA400083CA4000810
:105700003EA4000840A4000844A4000845A40008E2
:1057100046A4000847A4000848A4000849A40008BB
:105720004AA400084BA400084CA400084EA400089A
:105730004FA4000850A4000852A4000854A4000874
:1057400055A4000858A4000888A4000889A40008EB
:105750008AA400088CA400080021034A1160034AAF
:1057600011800180704700003400002038000020C4
:10577000002419E000BF00BFFCF7FAFC044600BF9C
:1057800000BF0A480068401C0849086008480068D3
:10579000401C0749086000BF00BF2046FCF7ECFC36
:1057A00000BF00BFFEF7E6FDE4E700002C0000208C
:1057B0006400002010B58AB0044600200E4908603D
:1057C0000B2000210591CDE90704069108460B49FD
:1057D00009680B4A12680B4B1B68CDE90132CDE911
:1057E00003103F200023084A08A100900C48FFF74F
:1057F000B1FA0AB010BD00002C000020A0A20008E1
:105800009CA2000898A200087157000875432F4F0A
:10581000532D4949492049646C65205461736B00DC
:10582000FC1100200021034A1160034A118001800D
:10583000704700003C0000204000002070B5014689
:105840001A4D2D681DB945F21E750D8070BD184D9D
:105850002D881DB945F21D750D80F7E7134D286899
:105860002A681032124D2D886D1EACB2002308E05C
:105870000260002545600581C560103010325D1C56
:10588000ABB2A342F4DB0025056045600581C5602D
:10589000064D2D68074E3560054D2D88B5800025D5
:1058A000F58035810D8000BFD0E70000D8A2000848
:1058B000D0A20008B012002010B5014648894B89DB
:1058C000002B17DD0A680C4B1B6813600A4C4B68F1
:1058D00023602346DB884C891B1B074CE38023464F
:1058E0009B884C892344044CA38000234B818B81EB
:1058F0000B604B6010BD0000B0120020018100223F
:1059000042818281026042607047000009A1C1614A
:10591000002141610849096811B90021816105E050
:1059200005490968816104490968486102490860BC
:105930007047000020000000440000200021034ABE
:105940001160034A1180018070470000440000206C
:10595000480000202DE9F04105460C4616461F463A
:105960001548006880F8346000201349096881F800
:10597000350039461048006800F050FC6CB104F165
:105980000808EC60012229460B48006800F016F870
:105990002946404600F08EF806E0002006490968D6
:1059A000C88705490968086303480168204600F074
:1059B00019F8BDE8F0810000BC00002010B5C287D6
:1059C000016300230AE000244C600C600C614C6110
:1059D0000C83CC61886020315C1CA3B29342F2DB63
:1059E00010BD000030B548B14568C1F8B05000F1B5
:1059F0000804226893681D6AC56113E091F8345069
:105A0000022D02D0072D08D103E007A5C1F8B05040
:105A100007E007A5C1F8B05003E008A5C1F8B050F1
:105A200000BF00BF30BD00005461736B2051000007
:105A30005461736B2053656D00000000200000006E
:105A400030B507A5C1F8B05000F1080422681AB1BA
:105A500093681D6AC56101E001A5C56130BD000004
:105A6000200000002DE9F04304460F4684F837700B
:105A7000256BB4F83E8013E0D5F80C9009F10806C8
:105A80003089012807D92946304600F05EF82946BA
:105A9000304600F00FF82035A8F101001FFA80F819
:105AA000B8F1000FE8D1BDE8F0830021016041604A
:105AB00001817047F0B58E6896F8375007893FB975
:105AC0000127078100274F600F600160416023E0DC
:105AD00007897F1C0781026806E0946894F8377094
:105AE000AF4200DD02E05268002AF6D100BF32B9B1
:105AF00000274F6043680B60596041600CE01768F5
:105B00002FB9116000270F604A60016004E013683C
:105B10000B604A6059601160F0BD2DE9F041044608
:105B2000256BE68F0AE0D5F80C8008F108072946B6
:105B3000384600F00AF82035701E86B2002EF2DCDE
:105B40000020E0872063BDE8F08110B50489012CB6
:105B500003D100240460446011E00C6824B94A6851
:105B60000024146002600AE04C6824B90B68002429
:105B70005C60436003E00B684A685A601360048904
:105B8000641E048100244C600C6010BD2DE9F843B4
:105B900006460C4617469846089D94F83600082895
:105BA0005BD2DFE800F0040508090607323300BFC6
:105BB00000BF00BF52E000BF94F83400032807D1B3
:105BC00043463A4621463046009500F04AF803E045
:105BD0002765A4F85480256436B12046FFF79DFF61
:105BE00021463046FFF72CFF94F83600032802D1F7
:105BF000204600F057FD204600F0AAF8002034347B
:105C0000A070607004F8340928E000BF94F83400F4
:105C1000032807D143463A4621463046009500F016
:105C200020F803E02765A4F85480256436B12046A7
:105C3000FFF773FF21463046FFF702FF94F8360066
:105C4000072802D1204600F02DFD04203434A07036
:105C50000020607004F8340900E000BF00BFBDE818
:105C6000F883F0B50446059E086BCD8F0AE0C7683F
:105C7000A74204D1046142610383C66104E020307D
:105C80006F1EBDB2002DF2DC00BFF0BD70B5002567
:105C9000074C03E005F12000C5B2241D2068002850
:105CA000F8D02068FCF76FFA2844C5B2284670BDCA
:105CB00008000020002004E00021034A42F82010E0
:105CC000401C0228F8D370470800002030B5420974
:105CD00000F01F030121C3F11F04A140034C54F83D
:105CE00022400C43014D45F8224030BD0800002001
:105CF00030B5420900F01F030121C3F11F04A14088
:105D0000034C54F822408C43014D45F8224030BDED
:105D1000080000200021034A1160034A118001801D
:105D200070470000500000205400002000210AE0CD
:105D300001EB4102054B03EB82000022028102606D
:105D400042604A1CD1B24029F2D37047BC120020F5
:105D500010B5044694F83700FFF7B8FF94F8370001
:105D600005490978884203D1204600F027F802E06F
:105D7000204600F003F810BD4A00002010B590F84E
:105D8000373003EB43030C4C04EB83010B893BB925
:105D900001230B810023C36003610860486009E0B0
:105DA0000B895B1C0B810B68C360002303610A68CD
:105DB0001061086010BD0000BC12002010B590F802
:105DC000373003EB43030B4C04EB83010B893BB9E6
:105DD00001230B810023C36003610860486008E071
:105DE0000B895B1C0B810023C3604A680261D06091
:105DF000486010BDBC1200202DE9F041054695F821
:105E0000370000EB4000124901EB80042F69EE6877
:105E100087B946B9002020812060606095F837007E
:105E2000FFF766FF0EE02089401E208100203061D0
:105E3000266007E02089401E2081FE600EB9676061
:105E400000E0376100202861E860BDE8F0810000D3
:105E5000BC1200200021034A1160034A1180018016
:105E600070470000580000205C00002086B0002031
:105E7000009006E0A7490968480001AA0021FFF741
:105E8000F3FAA54800780128F4D101A8FEF7CCFE6A
:105E90000027A24800689F490968884205D99F48A1
:105EA00000689C490968B0FBF1F727B99B48006876
:105EB0000A21B0FBF1F72BE14FF0000A00BF00BF51
:105EC000FCF756F9009000BF00BF9548006895495F
:105ED000086000209249086000BF00BF0098FCF7EE
:105EE0004BF900BF00BF904800688E49096888429E
:105EF00048D98D4800688D49884205D242F2107019
:105F000003900120029023E0874800688849884276
:105F100005D24FF47A7003900A20029018E082486C
:105F200000688449884203D26420039002900FE005
:105F30007D4800688049884205D20A2003904FF4CA
:105F40007A70029004E00120039042F210700290F7
:105F5000754801680298B1FBF0F972490398096825
:105F60004843B0FBF9F042F21071081A73490880F7
:105F7000734800880988884208DA704800887049A8
:105F8000088003E042F210706C490880FEF7D8FEEA
:105F9000002500BF00BFFCF7EBF8009000BF00BF7A
:105FA0006848046800BF00BF0098FCF7E5F800BF30
:105FB00000BF26E000BF00BFFCF7DAF8009000BF8A
:105FC00000BF54F8900F6060002044F8900900BFB3
:105FD00000BF0098FCF7D0F800BF00BFD4F89400D1
:105FE000054400BF00BFFCF7C3F8009000BF00BF2E
:105FF000D4F8AC4000BF00BF0098FCF7BDF800BF6C
:1060000000BF002CD6D145B34848854205D242F2A4
:10601000107005904FF0010B1BE04548854205D2FA
:106020004FF47A7005904FF00A0B12E04148854218
:1060300003D26420059083460BE03F48854204D29A
:106040000A2005904FF47A7B03E00120059042F28C
:10605000107BB5FBFBF0049003E0002005900120CD
:10606000049000BF00BFFCF783F8009000BF00BFA2
:106070003448046800BF00BF0098FCF77DF800BFFB
:1060800000BF2BE0D4F89400059948430499B0FB75
:10609000F1F086B242F21070864200D90646A4F8AA
:1060A0008060B4F88200B04201DAA4F8826001ABEB
:1060B00004F1A002111D2046FFF7DAF800BF00BF6F
:1060C000FCF756F8009000BF00BFD4F8AC4000BF0A
:1060D00000BF0098FCF750F800BF00BF002CD1D1E2
:1060E00019480078012805D100201749087001A837
:1060F000FEF79AFDCAF1000814480068404502D234
:106100001248C0F8008001AA00213846FFF7ACF918
:10611000D2E60000E0A2000870000020F8A200080B
:10612000640000206C00002068000020801A060037
:1061300000093D00005A62020084D7176000002069
:10614000620000207C0000205E000020740000201F
:1061500010B58AB0044600201F4908601F49086036
:106160001F4908601F4908701F4908701F480068D0
:1061700020B946F62B6020800AB010BD1C4800688C
:106180001C490968884203D246F62C602080F3E758
:10619000194800783F2803D346F62A602080EBE7B1
:1061A000032000210591CDE9070406910846104916
:1061B0000968124A12680D4B1B68CDE90132CDE91E
:1061C00003100D48007800230D4A0EA100901248DC
:1061D000FEF7C0FD00BFCFE7640000206C00002088
:1061E00068000020700000205E000020E4A200088B
:1061F000ECA20008F4A20008DCA20008E8A2000853
:106200006D5E000875432F4F532D49494920537443
:106210006174205461736B00BC15002070B5044696
:106220000D4645B12A462146064800F099F903205B
:1062300084F8360002E0022084F836002046FFF79A
:10624000DBFD70BD940000200021C0F8A8100949B2
:10625000096819B90021C0F8AC1007E005490968C0
:10626000C0F8AC1003490968C1F8A80001490860EA
:10627000704700007C000020D0F8A820D0F8AC10B7
:106280004AB90D4B196011B10023C1F8A8300023A1
:10629000C0F8AC300FE029B90023C2F8AC30C0F828
:1062A000A83008E0C2F8AC10C1F8A8200023C0F85C
:1062B000AC30C0F8A83070477C0000200021044AB0
:1062C0001160044A1180044A116001807047000087
:1062D0007C000020800000207800002070B504467B
:1062E00000202060A0606060E06020616061A061CB
:1062F000E06121A0206200206062A062E062206470
:106300002065A4F85400002104F15800FFF7F6FAC4
:106310000020A066E0666067A4F87C00A067002506
:1063200006E0002104F1700040F82510681CC5B299
:10633000002DF6D00020343420616066A0666060D5
:1063400084F84A002067E06620816061A061A4F8BB
:106350004C00A4F84E00206560650026A665E06547
:1063600020706070A0704020E07000206067A0671F
:1063700003A0E067343C70BD3F5461736B000000C4
:106380002000000008B504480068FEF75DFE69467D
:106390000020FEF7B9FD08BDBC0000202DE9F84340
:1063A0000446884617461D464FF0000900BF00BF4F
:1063B000FBF7DEFE814600BF00BF0CB967480468EA
:1063C00027640020288094F83600082876D2DFE879
:1063D00000F0040550510607525300BF00BF00BF34
:1063E0000420012804D0022813D0042833D122E04D
:1063F000606CFF280CD100BF00BF4846FBF7BCFE15
:1064000000BF00BF46F6C55028800020BDE8F883D5
:1064100022E04FF6FF71606C88420BD100BF00BFD5
:106420004846FBF7A9FE00BF00BF46F6C5502880CE
:106430000020EBE710E0606C401C58B900BF00BFC3
:106440004846FBF799FE00BF00BF46F6C5502880BE
:106450000020DBE700E000BF00BF606C401C606410
:10646000666C00BF00BF4846FBF786FE00BF00BF5A
:1064700071E000BF00BF00BF94F83400072815D1B9
:1064800000231A46214618460097FFF77FFB666CEB
:1064900000BF00BF4846FBF76FFE00BF00BF08F417
:1064A000004000284AD1FEF7BBFA47E0042001284B
:1064B00005D0022813D0042833D122E03FE0606CDD
:1064C000FF280BD100BF00BF4846FBF755FE00BFB9
:1064D00000BF46F6C5502880002097E722E04FF61F
:1064E000FF71606C88420BD100BF00BF4846FBF7CC
:1064F00043FE00BF00BF46F6C5502880002085E758
:1065000010E0606C401C58B900BF00BF4846FBF764
:1065100033FE00BF00BF46F6C5502880002075E757
:1065200000E000BF00BF606C401C6064666C00BF90
:1065300000BF4846FBF720FE00BF00BF0BE000BFD6
:1065400000BF4846FBF718FE00BF00BF46F62D60AF
:106550002880002600BF00BF304657E7BC0000205F
:1065600070B51546066846B98D6400264E618E6189
:10657000C86101600126868033E0046802682B460A
:1065800024E0966C9E421DD396696EB98B640026FA
:106590008E614A61C861966CF61A966491610160D9
:1065A0008688761C86800CE094698B648C614A61D5
:1065B000C861966CF61A9664916161618688761C52
:1065C000868070BD966C9B1B14465269002AD8D1F8
:1065D0008B648C6100264E61C86161618688761C7F
:1065E000868000BFEDE700002DE9F04104460D462E
:1065F00090461F46B8F1040F0ED1284800682E1AA5
:1066000016F5803F01D8002E3CD10020A06447F24F
:106610007E203880BDE8F081B8F1080F29D11F49EC
:10662000E06C0968081AA84205D92E461B48006884
:106630002844E06426E01949E06C0968081A2E1A1B
:1066400016F5803F00D886B91449E06C0968081A2D
:10665000B0FBF5F005FB0050E16C0844E06400205D
:10666000A06447F27E203880D4E7E06C2844E064E0
:1066700008E00DB12E4605E00020A06447F27E2020
:106680003880C7E7012084F83600324621460448A6
:10669000FFF766FF0020388000BFBBE784000020C2
:1066A0008C00002030B5C26983694169ABB929B952
:1066B0000024146094808464C4611EE000248C6112
:1066C0008C6C856C2C448C6411609488641E94805E
:1066D000002444618464C4610FE0596121B18B617D
:1066E0008C6C856C2C448C64002484619488641EBA
:1066F0009480002444618464C46130BD704700000C
:106700002DE9F0474FF0000900BF00BFFBF730FD57
:10671000814600BF00BF002700261C4D2C683CB3FB
:10672000A06C401EA0641FE0701C86B294F8360076
:10673000012806D1002084F836002046FFF708FB28
:1067400006E094F83600052802D1042084F83600CB
:10675000606928602C6814B90020A88007E0A88828
:10676000401EA8800020A061A06C0028DCD000BFE3
:10677000EE80C7F1000800BF00BF4846FBF7FCFCF5
:1067800000BF00BF4046BDE8F08700008C0000203D
:106790002DE9F0474FF0000900BF00BFFBF7E8FC10
:1067A000814600BF00BF00270026294D2C68002C21
:1067B00041D0A06C401EA06439E0701C86B294F8F1
:1067C0003600032813D100202065A4F8540020646B
:1067D0002046FFF7A2F92046FFF7BAFA002034342A
:1067E000A07003206070002004F8340913E094F8CE
:1067F000360007280FD100202065A4F8540020643B
:106800002046FFF78AF904203434A070032060701A
:10681000002004F83409606928602C6814B900204D
:10682000A88007E0A888401EA8800020A061A06C76
:106830000028C2D000BFEE80C7F1000800BF00BF33
:106840004846FBF799FC00BF00BF4046BDE8F08713
:10685000940000201CB500272CE001AB6A46002103
:106860000846FEF7FDFBBDF8040018BB124800788F
:1068700001281FD100BF00BFFBF77AFC074600BF0D
:1068800000BF0E480068401C0C49086000BF00BFF4
:106890003846FBF771FC00BF00BFFFF731FF06462B
:1068A000FFF776FF0546741905480068A04201D23B
:1068B00003480460D1E7000031000020840000207C
:1068C0008800002010B58AB00446002020490860E6
:1068D00020490860204908601E498880C8801E49F8
:1068E0008880C8801D48006820B947F212202080A7
:1068F0000AB010BD1A4800681A490968884203D2D4
:1069000047F213202080F3E7174800783F2803D38D
:1069100047F211202080EBE70B2000210591CDE903
:106920000704069108460E490A68104909680B4B8E
:106930001B68CDE90131CDE903200B480078002325
:106940000B4A0CA100901048FEF704FA00BFCFE7F5
:10695000840000208C0000209400002000A3000888
:1069600008A30008F4A20008FCA2000804A3000881
:106970005568000875432F4F532D494949205469E4
:10698000636B205461736B007016002010B58AB0E1
:10699000044600202F4908602F4908602F490880CD
:1069A0002F48006840B12F4800682D490968B0FBA6
:1069B000F1F02D49086006E02A4800680A21B0FB82
:1069C000F1F029490860284800682849086000203B
:1069D0002749086027490860224627A12A48FDF771
:1069E000FBFD208808B10AB010BD2848006818B91E
:1069F00047F247302080F6E72548006825490968B6
:106A0000884203D247F248302080ECE722480078E1
:106A10003F2803D347F246302080E4E70B200021D3
:106A200005910A46CDE907040691194800681B49FB
:106A30000968164B1B68CDE90131CDE90302164800
:106A400000780023164A17A100901C48FEF782F92F
:106A500000BFC8E79C000020A4000020A000002088
:106A600014A30008F8A20008B4000020B800002019
:106A7000B0000020AC0000204F5320546D72204D18
:106A800075746578000000002417002018A3000822
:106A900020A30008F4A2000810A300081CA300080B
:106AA000DD6A000875432F4F532D49494920546929
:106AB0006D6572205461736B000000005017002058
:106AC0000EB502A801AB0022114600900148FDF767
:106AD000C7FD0EBD24170020704700001CB53CE028
:106AE00001AB6A4600210846FEF7BAFAFFF7E8FF55
:106AF0004FF0000819480068401C18490860184801
:106B000004681EE001A8FDF7DBFF2769A069401EAD
:106B1000A061A06980B9A08C022802D1206AA0617E
:106B200005E0204600F020F8032084F82600A56840
:106B300015B12046E168A8473C4601A8FDF7F8FFDB
:106B400000BF002CDED1C8F1000600F02FF8054888
:106B50000068B04201D203480660C1E7B0000020DF
:106B6000A4000020AC00002010B50E4B1B6883422F
:106B700006D101690B4B196039B100234B6104E068
:106B8000416902690A6102B15161012380F826302E
:106B9000002303614361044B1B885B1E024C23806E
:106BA00010BD0000A4000020A000002008B56A4627
:106BB00000210248FDF77CFE08BD000024170020DC
:106BC0002DE9F05F04460D4690460027BA46BB46C5
:106BD000207810B12078012875D16078032806D07C
:106BE00064283BD0652874D066286ED1ADE0774824
:106BF000C0787649897800EB012087B273484079E4
:106C00007249097900EB01201FFA80FABAF10A0FE4
:106C100023DC0F2F21DC20782870032068704FEAD6
:106C20004A60000EA870FBF73FFF002610E0B8197D
:106C3000674931F8100001127000C01C2954B819BE
:106C4000634911F810107000001D2954701C86B2A1
:106C50005645ECDBA87800F1030BB0E0A7784FF6BF
:106C6000FF7000EA0727E07807435A48B0F842036C
:106C7000B8422BD101205749C8600020886100210B
:106C800054488183002604E0002153488155701C3C
:106C900086B2B6F5FA7FF7DB2078287060786870E6
:106CA000A078A870E078E870207928716079687120
:106CB0004FF0060BFCF788FC0020FCF779FC012064
:106CC0004649087004E07BE003E075E04FF0000BFC
:106CD00075E0B8F5837F35D13E48C068022831D1D0
:106CE00000203C498861A7784FF6FF7000EA07272B
:106CF000E078074301213848C1553648878300268C
:106D000006E0301D215C33481E308155701C86B270
:106D1000FF2EF6DD2F48D0F84C0320F00800083095
:106D20002C49C1F84C032078287060786870A078EE
:106D3000A870E078E87020792871607968714FF068
:106D4000060B01E04FF0000B39E0B8F1060F30D12F
:106D50002048C06802282CD100201E498861A778ED
:106D60004FF6FF7000EA0727E07807434FF000096D
:106D7000002606E01848805D48441FFA80F9701C20
:106D800086B2BE42F6DBB94504D1124887830320A0
:106D90001049C8602078287060786870A078A87062
:106DA000E078E87020792871607968714FF0060BFF
:106DB00001E04FF0000B02E04FF0000B00BF01E0DC
:106DC0004FF0000B5846BDE8F09F00002E30002029
:106DD0005C26002064190020AE1A0020C4000020A8
:106DE00010B50C4988690C49FBF79CFC06D20022BF
:106DF0004FF48051094802F069F80AE005498869B2
:106E00000749FBF785FC04D201221103034802F075
:106E10005DF810BD7821002000007A460010014086
:106E200000803B467047000010B50B49C8690B490C
:106E3000FBF778FC07D20848C069074908600220C0
:106E400081F8200006E004488069034908600120B9
:106E500081F8200010BD00007821002000803B4612
:106E600008B52648006840F001002449086000BFCA
:106E70002248006800F002000028F9D000BF1F4837
:106E8000406840F080001D4948600020009002E00A
:106E90000098401C009000985028F9D3174840688B
:106EA00040F09000154948600020009002E00098F2
:106EB000401C009000985028F9D300BF0F4840684C
:106EC00020F003000D494860084600680C4908405E
:106ED0000A4908604FF41F0088600846006820F4E3
:106EE0008020086000204860C86202F0BBFD4FF4BB
:106EF0000051880302F0ACF908BD00000010024008
:106F0000FFFFF6FE70B504462068012804D0022871
:106F100007D0032845D127E0FCF7BCFC0220206005
:106F200042E022488069401C204988610846806907
:106F30001F49884202D30020206014E01B4890F8CB
:106F40004C03C0F3C00070B172B61848D0F84C03BF
:106F500020F008001549C1F84C030846818B1E300B
:106F600000F012FA62B61FE0002020600F49898B02
:106F70000D0205EBD571491001F10A0000F0D8F9B6
:106F800000BFBFF34F8F0B48006800F4E0600A4970
:106F90000843001D07490860BFF34F8F00BF00BFC3
:106FA000FEE70020206000BF00BF70BD6419002014
:106FB000F82401000CED00E00000FA0510B50121F5
:106FC000344803F006F8012863D10121314802F06A
:106FD000FDFF0121304800F07DFF30480068401C73
:106FE0002E4908602E49884207D300202B490860AB
:106FF0002C480068401C2B49086028488088401CA9
:1070000080B226498880B0F57A6F28D30020888026
:10701000FCF75EF80446FBF711FB2349C860FCF758
:107020006FF80446FBF70AFB1F494860FCF75CF861
:107030000446FBF703FB1C49C861FCF76DF80446E6
:10704000FBF7FCFA1849886101F03CF8FCF7C2FA3A
:10705000154AD168106801F073FE01F04DFE0F482B
:10706000C088401C80B20D49C880B0F5C87F10D3DD
:107070000020C880FBF796FF0446FBF7DFFA0A49B9
:107080008860FBF74FFF0849486102F0EFFB01F011
:107090004DF910BD0034014000240140C80000201B
:1070A0007F1A0600DC0000207821002010B57A232A
:1070B000012290210148FDF727F810BDF82F00208C
:1070C00010B50A480A4908610015888240F2036039
:1070D000C86006484860C014088140F20360086038
:1070E0000846FCF704FFFFF7E1FF10BD000C01406C
:1070F000F82F002008B50020FCF75AFAFCF764FAD4
:10710000FBF7BEFD002000F08FF8002415E06A4672
:1071100000213220FEF7A8F9012204211D4801F0C8
:10712000D5FE6A4600213220FEF79EF90022042196
:10713000184801F0CBFE601CC4B2142CE7DB012020
:10714000FCF736FA24E014498868FBF7B2FA0446E3
:107150000B461148C16A224610A000F047F90E48BC
:107160002830FBF793FE0C482430FCF79BFDFCF71E
:10717000A5FC00F08BFFFFF757FEFFF731FEFBF792
:10718000EFFDFBF791FD6A4600210A20FEF76CF93E
:10719000D9E700000010014078210020493A256419
:1071A0002C252E30660A000010B50621184803F081
:1071B0001EF840B11749164803F03EF818B11549BA
:1071C000134803F030F81449114803F035F8F0B1D2
:1071D0000421124801F0E0F90F490D4803F023F8AB
:1071E0000B4802F0A3FF04210C4801F05EFBC0F540
:1071F000967421460A48FBF71DFE4FF4967204214F
:10720000064801F03FFB0421044801F0DEF910BDFF
:107210000038014006030600040304000000024099
:107220002E30002000BFFEE710B50446012C04D12B
:107230000221044801F048FE03E00221014801F068
:1072400041FE10BD001001402DE9F04704460F46F5
:107250009046A7EB08052846FBF7F0F9824621681F
:10726000FAF7F4FF8146FBF7F7F90646206AFBF7C9
:10727000E5F98146E169FBF74BFA07D2606AFBF753
:10728000DDF98146E169FBF74DFA13D3206AFBF77C
:10729000D5F98146E169FBF745FA01D8002D09DCF3
:1072A000606AFBF7CBF98146E169FBF731FA0DD84B
:1072B000002D0BDA2846FBF7C1F982466168FAF720
:1072C000C5FF81466169FAF769FF6061E06AFBF713
:1072D000B5F981466169FBF71BFA03D2E06AFBF757
:1072E000ADF96061A06AFBF7A9F981466169FBF716
:1072F00019FA03D2A06AFBF7A1F960613046FBF7E7
:107300009DF982466169FAF749FF8146FBF7A4F9C6
:107310000646606AB04200DA666A206AB04200DD62
:10732000266A3046FBF78AF9E0613046BDE8F0870F
:1073300010B5044601F036FC40F2053001F03EFB8A
:107340004FF4417001F03AFB40F2023001F036FB9D
:107350004AF6AA210B4801F041FB40F2053001F04A
:107360002DFB4FF4417001F029FB40F2023001F097
:1073700025FB21460348801C01F036FC01F08AFB06
:1073800010BD000000F0070870B505460E4601F07C
:1073900009FC40F2053001F011FB4FF4417001F09F
:1073A0000DFB40F2023001F009FB002417E00E4A09
:1073B000D31403FB0622022303FB042035F8141028
:1073C00001F00CFB40F2053001F0F8FA4FF4417087
:1073D00001F0F4FA40F2023001F0F0FA641C802C63
:1073E000E5D301F057FB70BD00A002080FB4054BB8
:1073F00010B503A9044A029800F0DAF810BC5DF851
:1074000014FB0000D58C0008B801002002E008C879
:10741000121F08C1002AFAD170477047002001E00E
:1074200001C1121F002AFBD1704700002DE9FF5F48
:1074300082B00021DDE90430020DDDF840B00343E5
:1074400018D044F61050A2F2FF324243151411989E
:1074500001281FD0A5EB0B00401C5FEA000A4FF08B
:1074600000064E4FDFF83891B046504615D5CAF1A8
:10747000000413E0119801244AA3012801D16FEA06
:107480000B010298119AC0E90031C0E9024206B02E
:10749000BDE8F09FCBF10000DFE704460021404A41
:1074A000491842EB0450CDE9001012E0E00707D084
:1074B00032463B4640464946FAF7DFFF804689465A
:1074C00032463B4610461946FAF7D7FF06460F46A6
:1074D0006410002CEAD1DDE90401DDE90023BAF1F2
:1074E000000F06DAFAF7C9FF42464B46FAF7C5FF26
:1074F00005E0FBF734F842464B46FBF730F804460C
:107500000E460022284BFBF72BFA03D84FF0FF3032
:10751000014607E00022254B20463146FAF706FFD8
:10752000FBF706FA102409E0002C0ADB0A220023EC
:10753000FBF718F9039B30321A55641E50EA01021A
:10754000F2D1641C039AC4F111031444119A012A64
:1075500003D0012208430DD10AE0084304D00020E3
:107560004FF0110B119072E7A3EB0B056D1E0DE0B0
:107570005B4504DD4FF0000205F1010504E003DA8C
:107580004FF00002A5F10105002AECD002981199F4
:10759000C0E90231C0E9004579E70000000014406D
:1075A0000000F03F300000000000F0430000E03F2A
:1075B0002DE9FF4F95B09B468946064600250FE210
:1075C000252877D100242746F84A0121059400E0B8
:1075D000044316F8013F203B01FA03F01042F7D1B3
:1075E00030782A2811D06FF02F033078A0F13002C4
:1075F000092A16D8059A44F0020402EB820203EB32
:1076000042021044761C0590EFE759F8042B0592CE
:10761000002A03DA504244F40054059044F0020476
:10762000761C30782E2816D116F8010F44F0040489
:107630002A280DD06FF02F023078A0F13003092BEB
:1076400009D807EB870302EB4303C718761CF3E75F
:1076500059F8047B761C30786C280FD006DC4C2857
:1076600017D068280DD06A2814D104E0742810D0EF
:107670007A280FD10DE044F400140AE044F4801499
:1076800001E044F440147278824202D104F580147F
:10769000761C761C307866280BD013DC582877D0FF
:1076A00009DC002875D04528F6D04628F4D04728B4
:1076B0001AD19DE118E0632835D0642879D0652877
:1076C00012D195E1702873D008DC6728F1D06928C1
:1076D0006FD06E280DD06F2806D1B5E073282CD05E
:1076E000752875D0782874D05A46179990476D1C24
:1076F00075E1C4F30250022809D003280DD0D9F84F
:10770000001004280DD00D6009F1040967E1D9F8D3
:107710000010EA17C1E90052F6E7D9F800100D8011
:10772000F2E70D70F0E719F8041B8DF80010002047
:107730008DF80100EA46012003E059F804AB4FF050
:10774000FF3061074FF0000102D40DE008F10101A4
:107750008846B9420FDA8045F8DB1AF8081000298C
:10776000F4D108E008F1010188468142FADB1AF8F9
:1077700008100029F6D105985B46A0EB08072146C2
:107780003846179A00F094FA284400EB080507E001
:107790004DE029E10DE01AF8010B5A461799904780
:1077A000B8F10108F7D25B4621463846179A13E133
:1077B00042E00A220092C4F302524FF0000A022A69
:1077C00008D059F804CB032A4FEAEC710AD00DE037
:1077D00029E02AE009F1070121F00702F2E802C1DD
:1077E000914609E00FFA8CFC4FEAEC71042A03D1B0
:1077F0004FFA8CFC4FEAEC71002907DA0A460021A7
:10780000DCF1000C61EB02012D2202E0220504D51F
:107810002B228DF80420012203E0E20701D0202270
:10782000F7E7904659E00A2102E010220DE010210E
:107830004FF0000A00910BE010224FF0000A44F0D4
:1078400004040827009203E008224FF0000A009287
:10785000C4F30252022A05D059F804CB0021032AAE
:1078600008D009E009F1070121F00702F2E802C19E
:10787000914605E01FFA8CFC042A01D10CF0FF0CA4
:107880004FF00008220728D5702806D0009B83F00F
:10789000100353EA0A0305D00EE040228DF80420BD
:1078A000012208E05CEA010206D030228DF80420B3
:1078B0008DF8050002229046009B83F0080353EAEE
:1078C0000A030AD15CEA010201D1620705D5302220
:1078D0008DF804204FF001087F1E582804D034A0F2
:1078E00003900EA802900DE036A0F9E753466046DB
:1078F000009AFAF737FF84460398825C0298401E8C
:10790000029002705CEA0100F0D1029806A9081A00
:1079100000F1200A600702D524F4803400E001273A
:10792000574502DDA7EB0A0000E0002000EB0A014A
:10793000009005984144401A0590E00306D45B4648
:107940002146179A059800F0B3F90544002706E090
:1079500001A85A46C05D179990476D1C7F1C47458A
:10796000F6DBE0030CD55B462146179A059800F03C
:107970009FF9054404E030205A46179990476D1C42
:107980000099481E00900029F5DC08E00298029951
:107990005A460078491C0291179990476D1CBAF11C
:1079A0000001AAF1010AF1DC65E1000009280100EB
:1079B0003031323334353637383961626364656665
:1079C0000000000030313233343536373839414227
:1079D000434445460000000000F058F90544761C79
:1079E000307800287FF4ECAD19B02846BDE8F08F60
:1079F000620700D4062709F1070222F0070CFCE811
:107A00000223E14603F000485FEA080C02D00FF2BF
:107A1000702C0DE05FEA045C02D50FF2682C07E0E1
:107A20005FEAC47C02D00FF2602C01E0AFF2700C70
:107A30004FF0FF3823F00043CDF850C065280CD03C
:107A400006DC452809D046281DD047283DD13DE019
:107A5000662818D067287ED138E00021112F01DB7D
:107A6000112000E0781CCDE9000106A90EA8FFF75F
:107A7000DDFCDDE90F010E9A03910021009207F170
:107A8000010A04914DE04FF000400097CDE901104C
:107A900006A90EA8FFF7CAFCDDE90F0203920E9BB0
:107AA00011990022DDF80CA00093049211B9791C01
:107AB00000EB010AB7EB0A0004D4C0F1FF3007F174
:107AC000010A0490AAEB0700019044E0012F00DABC
:107AD00001270021112F01DD112000E03846CDE9FA
:107AE000000106A90EA8FFF7A1FCDDE90F010E9A1F
:107AF0000391002104910092BA4621070CD4039906
:107B0000514500DA8A46BAF1010F05DD009AAAF163
:107B10000101515C302908D0B84202DA10F1040F9B
:107B200006DA0121CDE9011015E0AAF10101E9E72A
:107B3000002805DC049901440491AAEB000102E04D
:107B4000411C514500DD8A460499401A401C0190B1
:107B50004FF000400290200704D40198504501DB0B
:107B6000CDF8048000208DF84F0002980DF14F07EA
:107B7000B0F1004F25D02B200E9002984FF0020854
:107B800000280CDA404202902D200E9007E00A21D6
:107B90000298FAF7D1FD3031029007F8011DB8F1D3
:107BA0000001A8F10108F2DC02980028EFD1791E4B
:107BB0000E980870307800F0200040F0450007F87B
:107BC000020D12A8C01B00F107081498007800B13C
:107BD000012000EB0A01019801EBE0710598414496
:107BE000401A401E0590E00306D45B462146179AD2
:107BF000059800F05DF805441498007818B15A46CD
:107C0000179990476D1CE00324D55B462146179ACF
:107C1000059800F04DF805441CE00498002807DBA7
:107C2000DDE90301884203DD0098405C179901E01B
:107C3000179930205A469047049805F10105401CD9
:107C400004900198401E019004D12E205A461799A5
:107C500090476D1CBAF10001AAF1010ADDDC05E0D4
:107C600017F8010B5A46179990476D1CB8F100019F
:107C7000A8F10108F4DC5B462146179A0598ABE6AB
:107C80002D0000002B000000200000002DE9F04135
:107C9000044600251E461746880404D405E03946EC
:107CA0002020B0476D1C641EF9D52846BDE8F08140
:107CB0002DE9F041044600251E469046C80301D533
:107CC000302700E02027880404D505E041463846E7
:107CD000B0476D1C641EF9D52846BDE8F081816867
:107CE00041F00801816000BF816801F008010029AE
:107CF000FAD1816841F00401816000BF816801F020
:107D000004010029FAD1704730B5012902D00229B7
:107D10001AD10CE0C36A23F47003C362C36A541E11
:107D20004FF4700505EA04542343C3620DE0836BEE
:107D300023F440138363836B541E4FF4401505EA0C
:107D400004542343836300E000BF00BF30BD21B172
:107D5000826842F40062826003E0826822F400627A
:107D600082607047816841F48071816070478168EA
:107D700001F0010119B9816841F00101816070478A
:107D800072B101F001031BB1836843F48013836077
:107D900001F0020393B1836843F4004383600DE074
:107DA00001F001031BB1836823F48013836001F0A9
:107DB00002031BB1836823F40043836070470129E9
:107DC00002D0022910D107E0836823F46023836086
:107DD00083681343836008E0836823F4E04383608F
:107DE00083681343836000E000BF00BF7047CA434D
:107DF000026070470246002013680B4003B1012067
:107E0000704700000549096821F47021034A116098
:107E100011460968014311607047000004240140C5
:107E2000F0B51D4606290CD2436B01EB81071F26D6
:107E3000BE40B34301EB810602FA06F633434363C7
:107E400022E00C290ED2036B8E1F06EB86071F263D
:107E5000BE40B3438E1F06EB860602FA06F6334396
:107E6000036311E010290FD2C36AA1F10C0606EBDF
:107E700086071F26BE40B343A1F10C0606EB86061B
:107E800002FA06F63343C3620A2A0CD2046902EBF3
:107E900042070726BE40B44302EB420605FA06F647
:107EA0003443046111E0122A0FD2C468A2F10A0619
:107EB00006EB46070726BE40B443A2F10A0606EBCE
:107EC000460605FA06F63443C460F0BD0146C86CA8
:107ED00080B2704701F001021AB1826842F4800258
:107EE000826001F002021AB1826842F400128260DC
:107EF0007047AAB101F480731BB1436843F48073E7
:107F0000436001F480631BB1436843F480634360C2
:107F100001F00203CBB1836843F00203836014E0F5
:107F200001F480731BB1436823F48073436001F450
:107F300080631BB1436823F48063436001F0020354
:107F40001BB1836823F002038360704700B58BB0D8
:107F50000AA8032100220592CDE9062108901146C6
:107F60004FF480720848406E074BCDE90130CDE9EF
:107F7000032106200023054A05A100900948FCF7CB
:107F8000E9FE0BB000BD0000781D0020F570000870
:107F90005461736B204653424220436861726765A7
:107FA00000000000C41C002000B58BB00AA803210B
:107FB00000220592CDE90621089011464FF4807207
:107FC0000848406E074BCDE90130CDE9032105207B
:107FD0000023054A05A100900848FCF7BBFE0BB042
:107FE00000BD00005C220020E92B000841707020D9
:107FF0005461736B20436F6D6D000000A821002059
:1080000000B58BB00AA8032100220592CDE9062114
:10801000089011464FF480720848406E074BCDE936
:108020000130CDE903210D200023054A05A1009070
:108030000848FCF78FFE0BB000BD0000F82B0020B5
:10804000452C0008417070205461736B20574447E1
:1080500054000000442B002070B5044684F0010554
:108060002A460421014800F031FF70BD0010014094
:1080700010B500F017FF10BD10B504214FF41660C5
:1080800000F0DCFE00F016FF10BD000010B50B483C
:10809000407828B10A48007810B9FBF78FFA07E05A
:1080A0000648407820B90648007808B1FBF78CFAFA
:1080B000024840780249087010BD0000EC00002022
:1080C000D000002010B55B48407806287ED2DFE85B
:1080D00000F003043A526B91A9E0574890F82A0047
:1080E00078B15549C8685549FAF71CFB09D8524977
:1080F000C8685349FAF70CFB03D202204D49487077
:1081000020E04D4890F82A0078B14B49C8684C49A6
:10811000FAF708FB09D84849C8684A49FAF7F8FA53
:1081200003D20320434948700CE0434890F82A00EA
:1081300040B14149C8684349FAF7F4FA02D804202B
:108140003C49487073E03C49C8683D49FAF7EAFA8F
:1081500003D80320374948700CE0374890F82A00CC
:1081600028B13549C8683549FAF7D2FA02D2012058
:10817000304948705BE03049C8683349FAF7D2FAB1
:1081800003D804202B49487051E02B4890F82A006E
:1081900028B12949C8682949FAF7BAFA03D2012057
:1081A0002449487043E042E0234988682749FAF7A8
:1081B000AFFA05D82049C8682249FAF7B3FA07D9B7
:1081C0001D49C8682249FAF7ADFA00E02EE003D84D
:1081D0000520184948702AE0174890F82A0028B16D
:1081E0001549C8681549FAF793FA02D201201149D6
:1081F00048701CE000F00AFE03200E4908700E498A
:10820000C8681149FAF784FA08D80120094948706A
:108210001049087000201049086006E0064890F8F0
:108220002A0010B901200349487000E000BF00BFD8
:1082300010BD0000EC0000207821002000007A45ED
:108240000010A4460090E24600A8DE460000484325
:108250000078E646E0000020E400002010B50E495A
:10826000C8680E49FAF75EFA01D8012000E0002044
:10827000094981F82A00084690F82A0040B900F020
:10828000C5FD0320064908700020487005490870A4
:10829000014890F82A0010BD782100200000A0407D
:1082A000EC000020E800002010B501F0C5F840B156
:1082B00000F0ACFD00201249487003200870012036
:1082C00010BD01F099F890B901F074F878B901F097
:1082D0002FF860B901F00AF848B900F0C5FF30B9CD
:1082E00001F048F818B900F0E1FF0020E8E700F0DD
:1082F0008DFD002002494870032008700120DFE74F
:10830000EC00002070B506460D461446294630465E
:10831000FAF7FEF901D2284670BD21463046FAF739
:1083200001FA01D22046F7E73046F5E72DE9FC4196
:108330004D48807850B94C48407838B14A48407828
:10834000012803D048484078052801D1BDE8FC81C8
:108350004649C86AFAF772F90090454801680098E2
:10836000F9F76EFF20F0004442492046FAF7DAF9A7
:108370000FD20120404908700020404908603C4865
:1083800000683F4908603949C86AFAF757F93D491A
:1083900008603948007848B338480068401C3749BD
:1083A000086008460068C82806D3002032490870D3
:1083B00034480068009019E030480068FAF747F93F
:1083C00006462F4801682F480068F9F739FF07462D
:1083D0003146F9F73BFF05462649F9F769FF0446A0
:1083E000274801682046F9F7D9FE00902648007812
:1083F00040B326480068401C2449086008460068CD
:10840000FAF725F904462249FAF78CF908D8002032
:108410001D4908701549C86AFAF710F9009011E073
:108420001A480068FAF713F905461049C86AFAF7BE
:1084300005F906462946F9F709FF04461449F9F7F4
:1084400037FF00900A490098086008488268114880
:108450000099FBF79BF91049019008600198FBF720
:1084600049FA00BF72E70000EC00002078210020EC
:10847000B401002000004843A6010020A80100200C
:10848000AC010020B0010020E0000020E40000204A
:1084900000409C45F40000207C01002077E000BFF4
:1084A00000BF00BF00BF00BF00BF00BF00BF00BFD4
:1084B00000BF00BF00BF00BF00BF00BF00BF00BFC4
:1084C00000BF00BF00BF00BF00BF00BF00BF00BFB4
:1084D00000BF00BF00BF00BF00BF00BF00BF00BFA4
:1084E00000BF00BF00BF00BF00BF00BF00BF00BF94
:1084F00000BF00BF00BF00BF00BF00BF00BF00BF84
:1085000000BF00BF00BF00BF00BF00BF00BF00BF73
:1085100000BF00BF00BF00BF00BF00BF00BF00BF63
:1085200000BF00BF00BF00BF00BF00BF00BF00BF53
:1085300000BF00BF00BF00BF00BF00BF00BF00BF43
:1085400000BF00BF00BF00BF00BF00BF00BF00BF33
:1085500000BF00BF00BF00BF00BF00BF00BF00BF23
:1085600000BF00BF00BF00BF00BF00BF00BF00BF13
:1085700000BF00BF00BF00BF00BF00BF00BF00BF03
:1085800000BF00BF00BF00BF00BF00BF00BF011E93
:10859000A0F1010083D1704770B505460C46214615
:1085A000284600F063F908B900BFFEE704EB840039
:1085B000810005F10800405820F0010104EB84001F
:1085C000820005F10800815070BD70B505460C466B
:1085D0002146284600F04AF908B900BFFEE704EB3F
:1085E0008400810005F10800405840F0010104EBCF
:1085F0008400820005F10800815070BD70B5054609
:108600000C462146284600F031F908B900BFFEE7C4
:1086100004EB8400810005F10800405820F020019F
:1086200004EB8400820005F10800815070BD70B534
:1086300005460C462146284600F018F908B900BF47
:10864000FEE704EB8400810005F10800405840F08B
:10865000200104EB8400820005F10800815070BD08
:1086600000B587B04FF4A06000F0EAFF0421144881
:1086700000F02CF800208DF81A001248029001201A
:108680008DF81900002003904FF4967004900E4866
:10869000009000208DF8180001904FF44050059094
:1086A0006A460421064800F049F804210448FFF70F
:1086B000A5FF04210248FFF788FF07B000BD0000B6
:1086C000000002402E3000200438014070B50446FE
:1086D0000D462946204600F0C9F808B900BFFEE75C
:1086E00005EB8500810004F10800405820F00101ED
:1086F00005EB8500820004F108008150002105EBA4
:108700008500820004F10800815005EB850082009D
:1087100004F10C00815005EB8500820004F110008B
:10872000815005EB8500820004F1140081506068DF
:10873000AA000F2191400843606070BD2DE9F0410F
:1087400004460D4616462946204600F08FF808B923
:1087500000BFFEE705EB8500820004F110003168E0
:10876000815005EB8500820004F11400B16881504E
:10877000308A81B205EB8500820004F10C00815043
:1087800005EB8500810004F10800475827F47C5769
:10879000F1687068084371690843074305EB850079
:1087A000810004F108004750307E01280ED105EB0E
:1087B0008500810004F10800405840F0400105EBBD
:1087C0008500820004F1080081500DE005EB850072
:1087D000810004F10800405820F0400105EB8500BD
:1087E000820004F108008150707E01280ED105EB53
:1087F0008500810004F10800405840F0800105EB3D
:108800008500820004F1080081500DE005EB850031
:10881000810004F10800405820F0800105EB85003C
:10882000820004F108008150B07E70B905EB85002C
:10883000810004F10800405820F0100105EB85008C
:10884000820004F1080081500DE005EB85008100F5
:1088500004F10800405840F0100105EB850082004B
:1088600004F108008150BDE8F081000002460120BB
:10887000034B9A4202D1042900DD0020704700001A
:108880000004024070B506460C46154621463046A7
:10889000FFF7ECFF08B900BFFEE7A9B204EB8400C4
:1088A000820006F10C00815070BD70B505460C4683
:1088B00021462846FFF7DAFF08B900BFFEE704EBC0
:1088C0008400810005F10C00405870BD2DE9F04195
:1088D00005460026002700240EE005EB450000EBCE
:1088E000C5000A4A02EB8000001D50F824103046F3
:1088F000F9F754FC0646641C0A2CEEDB04493046AA
:10890000F9F7D6FC07463846BDE8F0810418002088
:108910000000204100B50346012200BF00F00CF822
:1089200002465B1E012A01D1002BF7D1012A00D19A
:108930000422104600BD000000200A49C96801F069
:10894000010109B101200CE00649C96801F01001DC
:1089500009B1032005E00349C96801F0040101B130
:10896000022070470020024000B50346012200BFEC
:1089700000F00CF802465B1E012A01D1002BF7D152
:10898000012A00D10422104600BD000000200A493F
:10899000C96C01F0010109B101200CE00649C96C64
:1089A00001F0100109B1032005E00349C96C01F091
:1089B000040101B10220704700200240064A02EB88
:1089C0009011096800F01F0301229A401143024BE5
:1089D00003EB9012116070470020024070B504460E
:1089E0000D46002627480088B0F5007F31D926487B
:1089F000844217D22548FFF78DFF0646002E3ED150
:108A00002348006940F001002149086125801F4882
:108A1000FFF780FF06461E48006920F001001C4950
:108A200008612CE01948FFF79FFF06463EBB184837
:108A3000006D40F001001649086525801348FFF7D6
:108A400093FF06461248006D20F0010010490865AA
:108A500015E00E48FFF75EFF064686B90C48006930
:108A600040F001000A49086125800848FFF752FFDD
:108A700006460748006920F00100054908613046B4
:108A800070BD0000E0F7FF1FFFFF07080000FF0FA9
:108A9000002002400848006940F080000649086153
:108AA00006480088B0F5007F04D90846006D40F004
:108AB000800008657047000000200240E0F7FF1FBB
:108AC00030B5054633480088B0F5007F44D93248B8
:108AD00085421CD23148FFF71DFF0446002C56D1B9
:108AE0002F48006940F002002D49086108464561A1
:108AF000006940F0400008612848FFF70BFF04467A
:108B00002748006920F00200254908613FE023481A
:108B1000FFF72AFF0446002C39D12148006D40F0B0
:108B200002001F49086508464565C06900F002005B
:108B300008B1084645611A48006D40F040001849E8
:108B400008651648FFF710FF04461548006D20F031
:108B50000200134908651AE01048FFF7DBFE0446DF
:108B6000ACB90F48006940F002000D4908610846A1
:108B70004561006940F0400008610848FFF7CAFEFF
:108B800004460748006920F00200054908612046B4
:108B900030BD0000E0F7FF1FFFFF07080000FF0FD8
:108BA000002002400C48006900F0800020B10B4812
:108BB000094948600A4848600A480088B0F5007FC3
:108BC00009D90548006D00F0800020B10348024932
:108BD0004864034848647047002002402301674509
:108BE000AB89EFCDE0F7FF1F70B504460D460026B8
:108BF00034480088B0F5007F43D93348844220D2FE
:108C00003248FFF787FE06463148006840F0020010
:108C10002F49FC39C1F8FC00002E51D108460069EB
:108C200040F00100086125602848FFF773FE064602
:108C30002748FC38006920F001002549FC3908610B
:108C40003EE02248FFF790FE06462148006840F0CB
:108C500002001F49FC39C1F8FC008EBB0846006DBC
:108C600040F00100086525601848FFF77DFE0646C4
:108C70001748FC38006D20F001001549FC390865E3
:108C80001EE01248FFF746FE06461148006840F015
:108C900002000F49FC39C1F8FC008EB90846006992
:108CA00040F00100086125600848FFF733FE0646E2
:108CB0000748FC38006920F001000549FC390861CB
:108CC000304670BDE0F7FF1FFFFF07080000FF0FF1
:108CD000FC20024070B504460D46E1B2054801F0A3
:108CE0002AFA00BF0721034801F081FA0028F9D0D1
:108CF000204670BD0038014010B5FFF7D5FA48B1E5
:108D000000F084F800200449C86203200349087079
:108D10000020487010BD000078210020EC000020E9
:108D200010B50021014801F068F910BD0034014080
:108D300010B50121014801F060F910BD0034014077
:108D40002DE9F04105460E462A4804782A488078E5
:108D500050B92A4890F82A0030B12748407818B115
:108D600025484078052801D1BDE8F08121480078E8
:108D700020B101280DD0022816D116E02049304636
:108D8000F9F70CFA07462946F9F7CCFC00D2022481
:108D900021E01B493046F9F753FA07462946F9F70F
:108DA000B7FC00D2022416E000BF16493046F9F79E
:108DB000F5F907462946F9F7ABFC01D2002409E092
:108DC00010493046F9F73CFA07462946F9F7AAFC5C
:108DD00000D2012400BF00BF07480078A04202D0A3
:108DE000012009490870044804700248047000BF5B
:108DF000BAE700006C010020EC0000207821002080
:108E000000803B4500007A456D01002010B5FAF75F
:108E10009BF9FFF785FF00221146064800F0E3FFAB
:108E200000220121034800F0DEFF00200249C86251
:108E300010BD0000003401407821002030B502460A
:108E40000B46164C002145F25550154D286000BFC9
:108E50001348C06800F00101601E041E01D0002903
:108E6000F6D109B1002030BD0D4843600B4C00BF66
:108E70000B48C06800F00201601E041E01D00029EA
:108E8000F6D109B10020EEE7C2F30B00044DA86053
:108E90004AF6AA2028600120E5E70000FFFF0F0046
:108EA000003000404AF6AA200149086070470000DF
:108EB000003000404CF6CC4001490860704700008B
:108EC0000030004041617047016170470AB10161A3
:108ED00000E041617047000010B540F2026000F010
:108EE000AFFB40F2046000F0ABFB40F2056000F025
:108EF000A7FB40F2066000F0A3FB4FF4805303226F
:108F000010211E4800F040F80423032210211C48C1
:108F100000F03AF84FF4805303221021184800F073
:108F200033F84FF4007303221021154800F02CF899
:108F30004FF4807303221021114800F025F8042318
:108F4000032210210F4800F01FF84FF400530322B2
:108F500048210B4800F018F800224FF480510748D0
:108F6000FFF7B4FFFAF7F0F8002000F0A7FD0122A8
:108F700004210448FFF7AAFF10BD000000080140CB
:108F80000010014000140140F0B5044616460025CB
:108F9000002201F00F0501F0100747B1042E05D1A2
:108FA00045F00305E76B1F43E76300E0354300200E
:108FB0001EE0012787401F40C7B122684FEA800C9E
:108FC0000F2707FA0CF7BA43870005FA07F73A4369
:108FD000282904D1012787401F40676105E04829FF
:108FE00003D1012787401F4027612260471CB8B288
:108FF0000828DED3082022E0012787401F40E7B180
:109000006268A0F108074FEA870C0F2707FA0CF7F0
:10901000BA43A0F10807BF0005FA07F73A43282929
:1090200004D1012787401F40676105E0482903D12B
:10903000012787401F4027616260471CB8B2102893
:10904000DAD3F0BD02469068084008B101207047AD
:109050000020FCE7F0B50A4600230024002100258B
:1090600000F00046B6F1004F02D11D4EF16901E05B
:109070001B4E7168C0F3034583B200F44016B6F589
:10908000401F08D121F0E061154E766826F0E066B9
:10909000134F7E6012E000F48016B6F5801F06D1F3
:1090A000032606FA05F4A14341F0E06106E0460D0F
:1090B000360103FA06F6B14341F0E06122B1460DF4
:1090C000360103FA06F6314300F00046B6F1004FD0
:1090D00002D1034EF16101E0014E7160F0BD00006C
:1090E00000000140C2680A400AB1416100E001612C
:1090F0007047000008B500F0B9FCFFF7EDFEFDF782
:10910000DFFFFAF74BFA00F085FF08A0FEF76EF9D3
:109110006846FBF739F9FEF747FFFEF717FFFEF742
:109120006FFF6846FBF74CFD002008BD0A0D205379
:10913000504D425F56322E3020757361727430206C
:109140007472616E736D6974207465737420210A82
:109150000D00000000B54FF480510248FFF7C2FF38
:1091600000BD00000008014010B5012200212520AB
:1091700000F002F810BD00002DE9F04103460D4655
:10918000164600240027A0462A48006800F4E06044
:10919000B0F5E06F03D100BF4FF0040830E0254880
:1091A000006800F4E060B0F5C06F03D101274FF014
:1091B000030825E01F48006800F4E060B0F5A06FE8
:1091C00002D10227B8461BE01A48006800F4E060AC
:1091D000B0F5806F03D103274FF0010810E0154868
:1091E000006800F4E060B0F5407F03D104274FF041
:1091F000000805E04FF4A06000F020F80227B84610
:10920000C7F1040005FA00F4C8F104010F20C840BA
:109210003040044324010848C45403F01F010120D6
:1092200088405911890001F1E021C1F80001BDE831
:10923000F08100000CED00E000E400E00249014391
:10924000024A1160704700000000FA050CED00E0D2
:10925000034A0A400243034B1A60BFF34F8F704723
:1092600080FFFF1F08ED00E010B50C49C8680C49ED
:10927000F9F74EFA0CD20B480078401CC0B20949ED
:109280000870052807DB052007498870012010BDFC
:109290000020044908700020F9E700007821002030
:1092A00000007A4598010020EC0000200D488078ED
:1092B00018B900200C49087070470B480078401C12
:1092C000C0B209490870052809DB002005498870EB
:1092D000012048700020044908700120ECE70020BC
:1092E000EAE70000EC0000209B01002010B50C49CB
:1092F00008680C49F9F716FA0CD20B480078401CA4
:10930000C0B209490870052807DB042007498870A6
:10931000012010BD0020044908700020F9E700007A
:109320007821002000E8004797010020EC00002091
:1093300010B50C4908680C49F9F7EAF90CD20B484A
:109340000078401CC0B209490870052807DB0320DB
:1093500007498870012010BD0020044908700020D2
:10936000F9E700007821002000803B4696010020AC
:10937000EC0000200C484069B0F5106F0FDD0B4881
:109380000078401CC0B2094908700A280ADD06208E
:1093900007498870002005490870012070470020A7
:1093A000024908700020F9E7782100209901002087
:1093B000EC00002010B50C4988680C49F9F7B2F9A7
:1093C0000CD20B480078401CC0B20949087005282F
:1093D00007DB022007498870012010BD00200449E6
:1093E00008700020F9E70000782100200080A244E6
:1093F00095010020EC00002010B50B4948680B498E
:10940000F9F790F90BD20A480078401CC0B208491D
:109410000870052806DB01200649887010BD002071
:10942000034908700020F9E7782100200060EA462F
:1094300094010020EC00002010B50C4988680C490C
:10944000F9F770F90CD20B480078401CC0B20949FA
:109450000870022807DB082007498870012010BD2A
:109460000020044908700020F9E70000782100205E
:109470000080A2449A010020EC000020184B59689B
:10948000184B1940164BDA6A22F000520C2820D2F1
:10949000DFE800F0060708091F0C1F0D1516171846
:1094A00000BF00BF00BF41EA803113E000BF20F0E1
:1094B00004004FF0805343EA803319430AE000BFB1
:1094C00000BF00BF20F00C0041EA803142F00052A2
:1094D00000E000BF00BF024B5960DA627047000035
:1094E00000100240FF3FFFEF2DE9F04F8CB0074620
:1094F00000200A904AA090E8004CC068CDE905BE63
:10950000CDF810A007900FF21C1ADAE9000ACDE995
:10951000020A0FF2101ADAE9000ACDE9000A4448FB
:109520004068C0F381000B900B9820B1012804D053
:1095300002283FD103E03F4A3EE03E4A3CE03C483F
:10954000406800F4803CBCF5803F12D13848C06AC6
:1095500000F08048B8F1000F01D1364B00E0364BE7
:109560003348406800F40039B9F5003F02D15B0888
:1095700000E0324B2E484068C0F383412C484068DD
:1095800000F0006008B141F010012948406800F087
:10959000804008B141F020010F2901D2891C06E06A
:1095A0000F2903D33E2901D8491C00E03F2103FBCA
:1095B00001F201E01F4A00BF00BF1D484068C0F330
:1095C000031504A8465D22FA06F419484068C0F362
:1095D000022502A8465D24FA06F009901448406866
:1095E000C0F3C2251DF8056024FA06F0089037B1D3
:1095F000012F06D0022F06D0032F0AD106E00A92CF
:1096000008E00A9406E009980A9003E008980A9096
:1096100000E000BF00BF0A980CB0BDE8F08F00006A
:109620000000000000000000010203040607080912
:109630000010024000127A00006CDC0200093D00BC
:10964000064A02EB9011096800F01F0301229A40BC
:109650001143024B03EB901211607047001002405F
:10966000064A02EB9011096800F01F0301229A409C
:109670009143024B03EB90121160704700100240BF
:10968000064A02EB9011096800F01F0301229A407C
:109690001143024B03EB901211607047001002401F
:1096A0002DE9F04105461948807818B100F0B4F86A
:1096B000BDE8F0814FF07A56154F324639462846BC
:1096C000FEF720FE054613492846F8F7BFFD804601
:1096D000F8F7DBFF84B24FF48E7200210E4800F0E1
:1096E00042FB224601210C4800F03DFB01220021F3
:1096F000094800F078FB01221146074800F073FB8F
:10970000FFF716FBF9F72AFD00BFD1E7EC000020B8
:109710000AD7233C008095430034014070B50546CC
:109720001348807810B100F077F870BD11492846D1
:10973000F8F78CFD0646F8F7A8FF84B22246002110
:109740000D4800F010FB0E2201210B4800F00BFB2E
:1097500001220021084800F046FB0122114606487C
:1097600000F041FBFFF7E4FAF9F7F8FC00BFDCE793
:10977000EC00002000809543003401402DE9F041C9
:1097800005460C461E48807818B100F045F8BDE843
:10979000F0811C4A1C492846FEF7B4FD05461B4AC9
:1097A00000212046FEF7AEFD044619492846F8F789
:1097B0004DFD0746F8F769FF86B23246002115488D
:1097C00000F0D1FA12492046F8F740FD0746F8F7B5
:1097D0005CFF86B2324601210E4800F0C4FA012235
:1097E00000210C4800F0FFFA01221146094800F060
:1097F000FAFAFFF79DFAF9F7B1FC00BFC7E70000DE
:10980000EC0000203333733F0AD7233CAE47613E60
:10981000008095430034014010B5002211460F48E6
:1098200000F0E1FA002211460C4800F09CFA0022F8
:1098300001210A4800F0D7FA00220121074800F070
:1098400092FAF9F781FC0020054948610320054997
:10985000087002200449087010BD00000034014067
:10986000F4000020EC0000206C01002010B52F480F
:10987000807828B100202E4908702E49087010BD4C
:10988000FEF7ECFC28B90020294908702949087026
:10989000F5E72948007848B9284890F82A0028B107
:1098A00001202749087000202649086021480078D7
:1098B00030B12249086824490968F8F729FF0AD21B
:1098C0001E4800682049086001201A4908700020DD
:1098D0001749087022E0194908681B490968F8F718
:1098E000AFFC04461949F8F71DFF14D21048007860
:1098F000401CC0B20E49087003280FDB012010493C
:10990000087000200F490860094908700B4800687A
:109910000D49086002E0002005490870074890F8EA
:109920002A000549087000BFA9E70000EC000020EC
:109930009C010020A4010020E800002078210020E4
:10994000E0000020E4000020A001002000409C4531
:10995000002000213F4A126842F480323D4B1A60D9
:1099600000BF401C3B4A126802F4003119B94FF69F
:10997000FF729042F5D1374A126802F400320AB9F8
:1099800000BFFEE7334AD26942F08052314BDA61C0
:10999000314A126842F440422F4B1A602D4A5268F5
:1099A0002C4B5A601A4652685A601A46526842F462
:1099B00080625A601A46526822F440325A601A464F
:1099C000526842F440325A601A465268234B1A4099
:1099D000204B5A601A465268214B1A431D4B5A605D
:1099E0001A46126842F080721A6000BF194A126863
:1099F00002F00072002AF9D0174A126842F480324D
:109A0000154B1A6000BF144A526802F48032002AD3
:109A1000F9D0114A126842F400320F4B1A6000BFAD
:109A20000D4A526802F40032002AF9D0094A5268FD
:109A300022F00302074B5A601A46526842F00202B3
:109A40005A6000BF034A526802F00802002AF9D0A7
:109A5000704700000010024000700040FFFFC3B7D5
:109A60000000340810B5FFF773FF10BD10B51248A1
:109A700000684FF47A71B0FBF1F4601EB0F1807FA2
:109A800001D301200FE0601E4FF0E02148610F215B
:109A90004FF0FF30FAF758FC00204FF0E0218861CA
:109AA00007200861002008B100BFFEE70021481E22
:109AB000FAF74AFC10BD00000000002010B5044673
:109AC00022464FF480510A48FFF700FA22464FF42D
:109AD00000710748FFF7FAF922464FF480710448F5
:109AE000FFF7F4F9224604210248FFF7EFF910BD11
:109AF0000010014000140140016841F08001016044
:109B000070470A884B881A438B881A43CB881A43BC
:109B10000B891A434B891A438B891A434264704755
:109B200010B531B101293FD002297DD003297CD164
:109B3000BFE0036A23F001030362836923F0030398
:109B40008361036A148823430362036A23F00203D8
:109B50000362036A9488234303626A4B984202D0EB
:109B6000694B98421FD1036A23F004030362036A1E
:109B7000548823430362036A23F008030362036AE1
:109B8000D48823430362436823F4807343604368AB
:109B9000148923434360436823F40073436043689C
:109BA000548923434360ABE0036A23F0100303624C
:109BB000836923F440738361036A148843EA0413BE
:109BC0000362036A23F020030362036A948843EA72
:109BD000041303624B4B984202D04B4B984226D160
:109BE000036A23F040030362036A548843EA0413C0
:109BF0000362036A23F080030362036AD48843EAA2
:109C000004130362436823F4806343604368148948
:109C100043EA84034360436823F40063436043687A
:109C2000548943EA840301E002E068E0436067E0AE
:109C3000036A23F480730362C36923F00303C361DF
:109C4000036A148843EA04230362036A23F400735B
:109C50000362036A948843EA04230362294B98420F
:109C600002D0294B984223D1036A23F48063036214
:109C7000036A548843EA04230362036A23F40063FB
:109C80000362036AD48843EA04230362436823F42B
:109C9000805343604368148943EA04134360436874
:109CA00023F4005343604368548943EA0413436038
:109CB00026E0036A23F480530362C36923F44073EC
:109CC000C361036A148843EA04330362036A23F41A
:109CD00000530362036A948843EA04330362094B26
:109CE000984202D0084B984208D1436823F480433D
:109CF00043604368148943EA8413436000E000BF73
:109D000000BF10BD002C01400034014031B10129D9
:109D10000CD0022913D0032922D118E0836923F043
:109D2000700383618369134383611AE0836923F4B9
:109D3000E0438361836943EA0223836111E0C369DD
:109D400023F07003C361C3691343C36109E0C369AE
:109D500023F4E043C361C36943EA0223C36100E023
:109D600000BF00BF704731B1012906D0022906D0DB
:109D7000032908D105E0426306E0826304E0C26380
:109D800002E0026400E000BF00BF704731B101296A
:109D90000CD0022913D0032922D118E0836923F0C3
:109DA000080383618369134383611AE0836923F4A1
:109DB00000638361836943EA0223836111E0C3691D
:109DC00023F00803C361C3691343C36109E0C36996
:109DD00023F40063C361C36943EA0223C36100E063
:109DE00000BF00BF704731B101290CD0022913D048
:109DF000032923D119E0036A23F001030362036AF4
:109E0000134303621BE0036A23F010030362036A37
:109E100043EA0213036212E0036A23F480730362CD
:109E2000036A43EA0223036209E0036A23F48053CE
:109E30000362036A43EA0233036200E000BF00BF2B
:109E40007047000010B504463349601A8C4244D074
:109E50000CDCB4F1804F1CD03048204410B3B0F576
:109E6000806F28D0B0F5006F52D12DE0B0F5806F33
:109E70003CD0B0F58E3F03D0B0F5923F48D13EE0E4
:109E800040F20B30FFF7FCFB40F20B30FFF7E8FB32
:109E90003FE04FF48060FFF7F3FB4FF48060FFF783
:109EA000DFFB36E040F20140FFF7EAFB40F2014001
:109EB000FFF7D6FB2DE040F20240FFF7E1FB40F256
:109EC0000240FFF7CDFB24E040F20340FFF7D8FB50
:109ED00040F20340FFF7C4FB1BE040F20440FFF7F1
:109EE000CFFB40F20440FFF7BBFB12E040F205401D
:109EF000FFF7C6FB40F20540FFF7B2FB09E040F276
:109F00000D30FFF7BDFB40F20D30FFF7A9FB00E07D
:109F100000BF00BF10BD00000010004000FCFFBFEC
:109F2000016841F001010160704700000A88826207
:109F30001D4A90420ED0B0F1804F0BD01B4A904288
:109F400008D01B4A904205D01A4A904202D01A4AC1
:109F500090420BD1026822F07002026002684B88C6
:109F60001A43026002688B881A4302608A68C262E0
:109F7000124A90420AD0124A904207D0026822F454
:109F8000407202600268CB881A430260064A90421F
:109F900002D0094A904201D10A7B0263426942F031
:109FA0000102426170470000002C014000040040A3
:109FB00000080040000C0040003401400010004048
:109FC00000140040C2680A43C2607047CA4302617D
:109FD00070470246D06800EA01031069084010B1DA
:109FE0000BB1012070470020FCE7426822F07002AC
:109FF000426042680A4342607047012904D1426CC2
:10A0000042F40042426403E0426C22F400424264A3
:10A010007047000010B5FFF7A7F8FEF721FB00F02E
:10A0200051F84FF44171024800F0F0F810BD000003
:10A03000003801402DE9F04704460D460027B84698
:10A04000B94600261D49601A8C421CD006DC1C480B
:10A05000204470B1B0F5806F1FD10FE0B0F5806F74
:10A0600016D0B0F56C4F18D10320FFF73DFA074624
:10A0700014E00220FFF738FA07460FE00220FFF74E
:10A0800033FA07460AE00220FFF72EFA074605E0FA
:10A090000220FFF729FA074600E000BF00BF07EBE8
:10A0A0005500B0FBF5F64FF6F07006EA000806F032
:10A0B0000F0948EA0900A060BDE8F087004C0040A5
:10A0C00000BCFFBF10B540F20260FFF7B9FA40F2E2
:10A0D0000E60FFF7B5FA4FF4007303221821114800
:10A0E000FEF752FF4FF48063032204210D48FEF770
:10A0F0004BFF0D4800F024F84FF4E1310A48FFF718
:10A1000099FF0421084800F0B3F80821064800F040
:10A11000B9F84021044800F05BF8034800F062F809
:10A1200010BD0000000801400038014001464868A9
:10A13000C0F308007047C1F3080242607047000096
:10A1400010B504462049601A8C4228D006DC1F480E
:10A15000204490B1B0F5806F33D117E0B0F5806F37
:10A1600026D0B0F56C4F2CD140F20E30FFF788FAB4
:10A1700040F20E30FFF774FA24E040F21140FFF78E
:10A180007FFA40F21140FFF76BFA1BE040F21240F9
:10A19000FFF776FA40F21240FFF762FA12E040F25F
:10A1A0001340FFF76DFA40F21340FFF759FA09E048
:10A1B00040F21440FFF764FA40F21440FFF750FAFF
:10A1C00000E000BF00BF10BD004C004000BCFFBF5E
:10A1D000426922F040024261426901F040031A43A1
:10A1E00042617047C16841F40051C160704710B5C9
:10A1F000024602EB9110006801F01F040123A34006
:10A20000184008B1012010BD0020FCE710B500EB9C
:10A210009112126801F01F040123A3401A4300EBBE
:10A2200091131A6010BDC1F3044301229A40D24336
:10A2300000EB91531A60704770B50246002300246A
:10A24000C1F38910105801F01F060125B54000EA3E
:10A25000050302EB91500068C1F304460125B540A7
:10A2600000EA050414B10BB1012070BD0020FCE729
:10A27000C26822F00402C260C26801F004031A43FB
:10A28000C2607047C26822F00802C260C26801F072
:10A2900008031A43C2607047BC0100200C00000094
:10A2A000800000000002000000000000000000002C
:10A2B000000000000000000000000000000000009E
:10A2C00000000000BC03002080000000000200002D
:10A2D0006400000040060000BC0500200A000000E9
:10A2E0000A000000FC0B00200C00000080000000B1
:10A2F0000002000040000000E80300000100000030
:10A30000FC0D00200C000000800000000002000096
:10A310000B00000064000000FC0F00200C00000097
:10A320008000000000020000401000000101010058
:10A330007856341201010000000000000000000007
:10A34000000000000000000000000000000000000D
:10A3500000000000000000000000000000000000FD
:10A3600001010100280004000000000000000000BE
:10A3700000000000000000000000000000000000DD
:10A3800000000000000000000000000001002000AC
:10A39000010010000C001000000000000000000090
:10A3A00000000000000000000000000000000000AD
:10A3B000000000000000000000000000000000009D
:10A3C00000000000010101002C00010020000C0031
:10A3D0002000400008000400000000000000000011
:10A3E000000000000000000000000000000000006D
:10A3F000000000000000000000000000000000005D
:10A400000000000000000000010101013000000018
:10A41000000000000000000000000000000000003C
:10A42000000000000000000000000000000000002C
:10A4300000000000000000000101010128000C00E4
:10A4400000030000040101010101010101000101FB
:10A45000B40008000101000000000000000000003E
:10A4600000000000000000000000000000000000EC
:10A4700000000000000000000000000000000000DC
:10A48000000000000000000001013000C176000063
:10A49000B1060000B4A4000800000020BC010000C8
:10A4A000D4290008E0A40008BC010020A433000067
:10A4B0001C74000805DD000E2707C2018203091D78
:10A4C0008FC2753C0AD7233C8202021302061D3F4D
:10A4D0006F12033B73E803F3E8030250020000002D
:04000005080021319D
:00000001FF
